:100000000C9445080C946D080C946D080C94680EC3
:100010000C94680E0C94680E0C946D080C946D088A
:100020000C946D080C946D080C946D080C946D087C
:100030000C946D080C946D080C946D080C946D086C
:100040000C941E0E0C946D080C941D0D0C94F70C62
:100050000C946D080C946D080C946D080C946D084C
:100060000C946D080C946D0800000000060001005F
:100070000002120803EF050006060801F00A000D51
:10008000100D00F124000B140D01EF4000141115A8
:1000900001F06B000E111001F0890002060501F05D
:1000A0008B0005170802EF9A0005170801EFA90059
:1000B00007070901EFB0000A0B0E02F6BE000206A8
:1000C0000702FFC00006020801F9C2000202060290
:1000D000FFC30007120700EFD3000B110D01F0EB77
:1000E0000005110D03F0F6000B110D01F00E010BD0
:1000F000110D01F026010B110D01F03E010B110D48
:1001000001F056010B110D01F06E010B110D01F004
:1001100086010B110D01F09E010B110D01F0B601CE
:10012000020D0602F4BA0102100602F5BE010C0C23
:100130000E01F5D0010C060E01F8D9010C0C0E01D0
:10014000F5EB010A120D02EF020216151801EF3C41
:100150000210121000EF60020D121002EF7E020F6B
:10016000121101EFA0020E121102EFC0020C120FC9
:1001700002EFDB020B120E02EFF40210121201EF7B
:1001800018030D121102EF360302120702EF3B03B0
:1001900009120D01EF50030E121002EF70030A1244
:1001A0000E02EF870310121402EFAB030D121202BE
:1001B000EFC90311121301EFF0030C121002EF0B41
:1001C0000411131301EF34040E121102EF54040E44
:1001D000121001EF74040C120F01EF8F040D1211B5
:1001E00002EFAD040F120F00EFCF0416121600EF4E
:1001F00001050F121000EF230510121000EF470544
:100200000D120F01EF650504170702EF71050712C4
:100210000700EF810504170701EF8D0509090B01A0
:10022000F098050F010DFF049A0505040601EF9DE6
:10023000050C0D0D01F4B1050C120D01EFCC050AF2
:100240000D0C01F4DD050B120D01EFF6050B0D0D84
:1002500001F4080605120701EF14060B120D01F454
:100260002D060A120D01EF440602120502EF49069F
:1002700004170600EF55060B120C01EF6E06021272
:100280000501EF7306110D1301F48F060A0D0D0120
:10029000F4A0060B0D0D01F4B2060C110D01F4CC07
:1002A000060B110D01F4E406060D0801F4EE060A32
:1002B0000D0C01F4FF0605100701F109070A0D0DE9
:1002C00001F41A070C0D0C00F42E07110D1100F4A7
:1002D0004A070B0D0B00F45C070B120B00F47507BB
:1002E0000A0D0C01F4860705170801EF95070217A0
:1002F0000602EF9B0705170802EFAA070A050C0183
:10030000F6FFFFFFF0F0CF3CF38A200630310318F0
:1003100018C7FFBFFC31031818C7FFBFFC31011815
:1003200018C0C606300403E1FF726C4788F107204D
:100330007E03F017023C4788F11B267FC3E01002C2
:1003400000000603C0407E0C0E7080C3180C310004
:10035000E73007E6003C40000C7C008FE019C70145
:1003600018303183021C7040FE0407C00F007E036A
:100370009C0C3030C0E701F803803E01CC6E19B010
:100380007CC0F303CE1F9FE61E1CFFA0088C6631C5
:1003900098C6318C63086308610C208218C318C3A7
:1003A00018C6318C623188C4620010235BE38D91E2
:1003B000000C0300C030FFFFF0C0300C0300C0F59C
:1003C00060FFF0F0020C1020C1020C1020C1020CE2
:1003D0001020C1001F07F1C7306E0F80F01E03C050
:1003E000780F01E03C0EC19C71FC1F0008CFFF8C10
:1003F0006318C6318C63181F0FF987607C0600C034
:10040000180701C0F0781C0600803007FFFFE03FAE
:100410000FF387606C0C0180707C0F801801803CAA
:100420000780D873FC1F000180700E03C0D81B0624
:10043000618C218C33067FFFFE0300600C01803F3E
:10044000CFF980300600DE1FE70E00E00C0180309F
:100450000781F873FC1F000F07F9C3307401803364
:10046000C7FEF0DC1F01E03C06C1DC71FC1F00FF91
:10047000FFFC010060180200C0300601803004015A
:10048000803006018030001F07F1C730660CC18C38
:1004900061FC3F8E3B01E03C0780D831FC1F001F10
:1004A00007F1C7706C0780F01E0761EFFC798030A0
:1004B00005819873FC1E00F00003C0F0000F560089
:1004C000000701E0F83C0F00E007C00F003C00F01F
:1004D00001FFFFFF000000FFFFFF000E007801F0AA
:1004E00007C00F00701E0F03C0F008001F1FEE1B97
:1004F00003C0C0300C060381C0E0300C03000000D4
:100500000C030000FE000FFE00F03E07003C380028
:1005100030C1E0660FD9D861C3C3070F1C1C3C6013
:1005200060F18183C6061B1838EE71E718FDF8717B
:10053000E7C0E00001E00001FFC001FC0003C003D0
:10054000C003C007E0066006600E700C300C301C63
:100550003818181FF83FFC301C300C700E60066015
:1005600006FFC7FF3019806C03601B00D80CFFC763
:10057000FF300D803C01E00F007806FFF7FE00071A
:10058000E03FF0E0738066006C0030006000C00166
:10059000800300060006006C00DC031E0E1FF80F2F
:1005A000C0FF83FF8C07300EC01B007C00F003C02F
:1005B0000F003C00F003C01F006C03B01CFFE3FF02
:1005C00000FFFFFFC00C00C00C00C00C00FFEFFEDE
:1005D000C00C00C00C00C00C00FFFFFFFFFFFF00BD
:1005E000600C0180300600FFDFFB00600C018030F2
:1005F0000600C0180007F01FFC3C1E70066003E0F8
:1006000000C000C000C07FC07FC003C003600360A3
:1006100007300F3C1F1FFB07E1C01E00F007803CA6
:1006200001E00F007803FFFFFFF007803C01E00FBF
:10063000007803C01E00C0FFFFFFFFF00180C06014
:1006400030180C06030180C0603C1E0F07C77F1FD7
:1006500000C03B01CC0E3070C3831C0CE03380DE45
:1006600003DC0E383060C1C3038C06301CC03B0075
:1006700060C0300C0300C0300C0300C0300C03001D
:10068000C0300C0300FFFFF0E007E007F00FF00FB1
:10069000D00FD81BD81BD81BCC33CC33CC33C6637C
:1006A000C663C663C3C3C3C3C3C3C183E01F00FC27
:1006B00007E03D81EE0F3079C3C61E18F0E7833C9A
:1006C0001DE06F01F80FC03E01C003E00FFC0F07F3
:1006D0008600C60033001B00078003C001E000F065
:1006E0000078003600330018C018783C1FFC03F86F
:1006F00000FF8FFEC06C03C03C03C03C07FFEFFC53
:10070000C00C00C00C00C00C00C00C0003E00FFCCB
:100710000F078600C60033001B00078003C001E0FE
:1007200000F00078003600330198C0FC783C1FFFD1
:1007300003F9800040FFC3FFCC03B006C01B006C70
:1007400001B00CFFE3FFCC03B006C01B006C01B08E
:1007500006C01B00700FE07FC3839C07600D8006FE
:10076000001E003F803FC00F8007C00F003E00DE2C
:100770000E3FF03F80FFFFFF0600600600600600AE
:10078000600600600600600600600600600600600B
:10079000C01E00F007803C01E00F007803C01E007F
:1007A000F007803C01E00F80EE0E3FE07C00600629
:1007B000C01DC031806301C70306060C1C1C301825
:1007C0006031C073006600DC01F001E003C0070087
:1007D000E0301D80E0760781D81E06707C18C1B01D
:1007E000E30CC38C330C38C6306718C198670661B8
:1007F000D81D83603C0D80F03E03C0700F01C0180F
:100800000700700E6038E060E1C0C301CC01F80160
:10081000E0038007801F003300E70386060E1C0EEE
:10082000700CC01C6006700E301C38181C380C3060
:100830000E70066003C003C001800180018001804A
:100840000180018001800180FFFFFFC00E00E00EEB
:10085000006007007007003003803803801801C073
:100860001C00FFFFFFC0FFCCCCCCCCCCCCCCCCCC84
:10087000CFF08181020604081810206040818102B7
:100880000604FF3333333333333333333FF00C0E4B
:100890000586C321198C83C180FFFEE38C303F079E
:1008A000F8E1CC0C00C01C3FCF8CC0CC0CE3C7EFF0
:1008B0003C70C00C00C00C00C00CF8DFCF0EE07C18
:1008C00003C03C03C03C03E06F0EDFCCF81F0FE712
:1008D0001B83C0300C0300C038371CFE1F000060B3
:1008E0000C018030063CCFFB8FE0F80F01E03C07A5
:1008F00080F83B8F3F63CC1F07F1C7703C07FFFFB9
:10090000FE00C01C0DC31FE1F03BD8C67FEC63188E
:10091000C6318C63001E67FDC7F07C0780F01E03A4
:10092000C07C1DC79FB1E600C03E0E7FC7E0C0304F
:100930000C0300C033CDFBC7E0F03C0F03C0F03C1C
:100940000F03C0F030F03FFFFFF0330003333333C9
:10095000333333333FE0C0180300600C018330C6EB
:1009600030CC1B83F0770C618E30E60CC1D818FFB9
:10097000FFFFFFF0CF1F6FDFFC78FC183C0C1E065A
:100980000F03078183C0C1E060F03078183C0C1879
:10099000CF37EF1F83C0F03C0F03C0F03C0F03C004
:1009A000C01F07F1C7707C0780F01E03C07C1DC705
:1009B0001FC1F0CF8DFCF0EE06C03C03C03C03C06D
:1009C0003E07F0EFFCCF8C00C00C00C0001E67FD9E
:1009D000C7F07C0780F01E03C07C1DC79FF1E600B6
:1009E000C018030060CF7F38C30C30C30C30C03E4A
:1009F0001FEE1B00C03C07F03E01F03E1DFE3E0016
:100A00006319FFB18C6318C631E7C0F03C0F03C017
:100A1000F03C0F03C0F07E3DFB3CC0E06606606723
:100A20000C30C30C3981981981F00F00E00E00C121
:100A3000C1B0E1D870CC2C6636319B18CD98646C6F
:100A400016360F1A078F038380C1C060EE18C60CDC
:100A5000C1F01C0180781B0330C7306606E06C0DC6
:100A60008338630C630E60CC1B03603C0700E01806
:100A70000300E0780E00FFFFF0180C070381C06050
:100A800030180E03FFFFC019CC6318C631998618C1
:100A9000C6318C631C60FFFFFFFFFFFCC718C63127
:100AA0008C630C33318C6318C67300703E09E41FED
:100AB000038000000000240027002A0004E0100248
:100AC0001C07123732292D29252B3900010310E18B
:100AD00010031D07062E2C292D2E2E373F00000255
:100AE0001013800A298064022A040000007F2B046E
:100AF0000000009F0F0180961180FFB103012C2D93
:100B0000B203012C2DB306012C2D012C2DB40107AD
:100B1000C003A20284C101C5C2020A00C3028A2A1C
:100B2000C4028AEEC5010E20003601C83A01050153
:100B3000036800207E1D00000000003E5B4F5B3E0E
:100B40003E6B4F6B3E1C3E7C3E1C183C7E3C181C92
:100B5000577D571C1C5E7F5E1C00183C1800FFE789
:100B6000C3E7FF0018241800FFE7DBE7FF30483A2F
:100B7000060E2629792926407F050507407F052591
:100B80003F5A3CE73C5A7F3E1C1C08081C1C3E7F19
:100B900014227F22145F5F005F5F06097F017F00E0
:100BA0006689956A606060606094A2FFA294080400
:100BB0007E040810207E201008082A1C08081C2A21
:100BC00008081E101010100C1E0C1E0C30383E3879
:100BD00030060E3E0E06000000000000005F000020
:100BE0000007000700147F147F14242A7F2A122391
:100BF0001308646236495620500008070300001CA1
:100C00002241000041221C002A1C7F1C2A08083EA9
:100C100008080080703000080808080800006060BC
:100C20000020100804023E5149453E00427F40002A
:100C300072494949462141494D331814127F102702
:100C4000454545393C4A4949314121110907364951
:100C5000494936464949291E000014000000403425
:100C6000000000081422411414141414004122142A
:100C70000802015909063E415D594E7C1211127C51
:100C80007F494949363E414141227F4141413E7FB2
:100C9000494949417F090909013E414151737F0892
:100CA00008087F00417F41002040413F017F081438
:100CB00022417F404040407F021C027F7F04081099
:100CC0007F3E4141413E7F090909063E4151215E77
:100CD0007F09192946264949493203017F01033F0B
:100CE0004040403F1F2040201F3F4038403F63149A
:100CF00008146303047804036159494D43007F419C
:100D000041410204081020004141417F04020102D8
:100D100004404040404000030708002054547840FD
:100D20007F284444383844444428384444287F3891
:100D30005454541800087E090218A4A49C787F0813
:100D400004047800447D40002040403D007F10288E
:100D5000440000417F40007C047804787C0804044F
:100D6000783844444438FC1824241818242418FCE7
:100D70007C08040408485454542404043F44243C8C
:100D80004040207C1C2040201C3C4030403C4428FB
:100D90001028444C9090907C4464544C4400083695
:100DA0004100000077000000413608000201020403
:100DB000023C2623263C1EA1A161123A4040207A23
:100DC000385454555921555579412254547842216B
:100DD0005554784020545579400C1E5272123955A2
:100DE000555559395454545939555454580000459F
:100DF0007C410002457D420001457C407D1211127C
:100E00007DF0282528F07C545545002054547C540E
:100E10007C0A097F4932494949323A4444443A32CA
:100E20004A4848303A4141217A3A42402078009D70
:100E3000A0A07D3D4242423D3D4040403D3C24FF1C
:100E40002424487E4943662B2FFC2F2BFF0929F6CB
:100E500020C0887E090320545479410000447D411C
:100E60003048484A32384040227A007A0A0A727D75
:100E70000D19317D2629292F282629292926304890
:100E80004D4020380808080808080808382F10C8FE
:100E9000ACBA2F102834FA00007B000008142A1482
:100EA0002222142A14085500550055AA55AA55AAFD
:100EB000FF55FF55FF000000FF00101010FF001449
:100EC0001414FF001010FF00FF1010F010F01414A5
:100ED00014FC001414F700FF0000FF00FF1414F4CA
:100EE00004FC141417101F10101F101F1414141FCB
:100EF00000101010F0000000001F101010101F1044
:100F0000101010F010000000FF1010101010101042
:100F10001010FF10000000FF140000FF00FF000091
:100F20001F10170000FC04F414141710171414F405
:100F300004F40000FF00F714141414141414F70040
:100F4000F7141414171410101F101F141414F41491
:100F50001010F010F000001F101F0000001F140000
:100F60000000FC140000F010F01010FF10FF14142B
:100F700014FF141010101F00000000F010FFFFFFFE
:100F8000FFFFF0F0F0F0F0FFFFFF0000000000FFB7
:100F9000FF0F0F0F0F0F3844443844FC4A4A4A34BD
:100FA0007E02020606027E027E02635549416338D4
:100FB00044443C04407E201E2006027E020299A585
:100FC000E7A5991C2A492A1C4C7201724C304A4DE3
:100FD0004D303048784830BC625A463D3E49494918
:100FE000007E0101017E2A2A2A2A2A44445F4444C1
:100FF00040514A444040444A51400000FF0103E050
:1010000080FF000008086B6B083612362436060F86
:10101000090F06000018180000001010003040FFF3
:101020000101001F01011E00191D1712003C3C3C6C
:101030003C00000000000000000800020100000366
:101040000407000000000000000000000000250070
:1010500028002B00000000002300260029000404C3
:101060000404040404040202020202020303030350
:10107000030301020408102040800102040810202C
:1010800001020408102035312B3111241FBECFEF8F
:10109000D8E0DEBFCDBF13E0A0E0B1E0E6EEF1E7BF
:1010A00002C005900D92A232B107D9F724E0A2E266
:1010B000B3E001C01D92A139B207E1F718E0C4E422
:1010C000D8E004C02197FE010E94DB38C334D10769
:1010D000C9F70E9439190C94E6380C940000CF929D
:1010E000DF92EF92FF920F931F93CF93DF936C01E8
:1010F0007A018B01C0E0D0E0CE15DF0589F0D80180
:101100006D918D01D601ED91FC910190F081E02D62
:10111000C6010995892B11F47E0102C02196ECCFFE
:10112000C701DF91CF911F910F91FF90EF90DF905A
:10113000CF900895FC01538D448D252F30E0842FEE
:1011400090E0821B930B541710F0CF9608950197EF
:101150000895FC01918D828D981761F0828DDF01D9
:10116000A80FB11D5D968C91928D9F5F9F73928F9A
:1011700090E008958FEF9FEF0895FC01918D828D8F
:10118000981731F0828DE80FF11D858D90E008955C
:101190008FEF9FEF0895FC01918D228D892F90E0B4
:1011A000805C9F4F821B91098F739927089581EA74
:1011B00093E00E94CB0821E0892B09F420E0822FE4
:1011C0000895FC01848DDF01A80FB11DA35ABF4F04
:1011D0002C91848D90E001968F739927848FA68936
:1011E000B7892C93A089B1898C9180648C93938D5D
:1011F000848D981306C00288F389E02D80818F7D4D
:1012000080830895EF92FF920F931F93CF93DF9304
:10121000EC0181E0888F9B8D8C8D981305C0E88947
:10122000F989808185FD24C0F62E0B8D10E00F5FBB
:101230001F4F0F731127E02E8C8DE8120CC00FB6D4
:1012400007FCFACFE889F989808185FFF5CFCE01C7
:101250000E94E108F1CF8B8DFE01E80FF11DE35AEA
:10126000FF4FF0820B8FEA89FB898081806207C083
:10127000EE89FF896083E889F989808180648083B1
:1012800081E090E0DF91CF911F910F91FF90EF905F
:101290000895CF93DF93EC01888D8823C9F0EA8904
:1012A000FB89808185FD05C0A889B9898C9186FD5F
:1012B0000FC00FB607FCF5CF808185FFF2CFA8895C
:1012C000B9898C9185FFEDCFCE010E94E108E7CF6F
:1012D000DF91CF91089580E090E0892B29F00E9462
:1012E000D70881110C9400000895833081F028F410
:1012F000813099F08230A1F008958730A9F08830CC
:10130000B9F08430D1F4809180008F7D03C080914A
:1013100080008F7780938000089584B58F7702C016
:1013200084B58F7D84BD08958091B0008F7703C010
:101330008091B0008F7D8093B00008953FB7F894FE
:101340008091990390919A03A0919B03B0919C0383
:1013500026B5A89B05C02F3F19F00196A11DB11D10
:101360003FBFBA2FA92F982F8827820F911DA11D4B
:10137000B11DBC01CD0142E0660F771F881F991F88
:101380004A95D1F7089520919F033091A003281723
:10139000390771F490919D0380919E03981741F055
:1013A000E0919D03F0E0E85AFC4F808190E00895C1
:1013B0008FEF9FEF089508951F93CF93DF93DC0184
:1013C0005C962D913C915D972115310539F481E0B2
:1013D00090E013969C938E9312973DC05196ED9199
:1013E000FC91529750969C915097892F80951FB7EA
:1013F0005E964C915E9741FB772770F941FD6095B1
:10140000F8944081772311F0492B01C04823408391
:10141000E9012197F1F748E0508160FF02C0592BA4
:1014200001C058235083E9012197F1F76695415097
:1014300099F7772321F090818923808303C08081ED
:10144000982B90831FBF5C968D919C915D9701971F
:10145000F1F721E030E0C901DF91CF911F910895AC
:1014600020919F033091A0032817390771F48091D0
:101470009E0320919D0390E0805C9F4F821B910909
:1014800060E470E00E947238089580E090E0089572
:1014900020919F033091A00328173907B9F4909148
:1014A0009D0380919E03981789F0E0919D03F0E0E1
:1014B000E85AFC4F808120919D0330E02F5F3F4F21
:1014C0002F73332720939D0390E008958FEF9FEFB4
:1014D0000895EF92FF920F931F93DC01ED91FC9121
:1014E00011971A960D911C911B9718962D913C916E
:1014F000199700A0F1A1E02D7B0140E050E060E0F1
:1015000070E009951F910F91FF90EF9008950E9450
:10151000E138611102C060E201C061E20C940F1574
:101520001F93CF93DF93EC01162F66E30E940F15F4
:10153000612F63706D8B8A8D623089F16330A9F100
:101540006130D1F0823011F460EC01C068ECCE0162
:101550000E94D71480E890E0998788878A8D81302F
:1015600019F480E890E002C080EA90E09B878A87C7
:10157000DF91CF911F910895823011F460EA01C08C
:1015800068EACE010E94D7148A8D813019F480E870
:1015900090E002C080EA90E099878887E2CF8230AD
:1015A00011F460E0D4CF68E0D2CF823011F460E66D
:1015B000E8CF68E6E6CFAF92BF92CF92DF92EF928C
:1015C000FF920F931F93CF93DF93EC0159016801B2
:1015D00028853985621773070CF05CC08A859B8566
:1015E000481759070CF056C0FB01EA0DFB1D2E17DA
:1015F0003F071CF45901A61AB70A9A012C0D3D1D8C
:10160000821793071CF46C01C41AD50A0FEF040F5C
:101610000C0D2FEF260F2A0DCE010E944815809148
:101620003E0490913F040E94D414EAA1FBA1908152
:101630008CA5892B8083E8A1F9A190818BA5809549
:10164000892380831C141D049CF485011016110647
:101650005CF46F2DCE010E94A6146E2DCE010E9467
:10166000A61401501109F2CF81E0C81AD108EACFBF
:10167000E8A1F9A190818BA5892B8083DF91CF917F
:101680001F910F91FF90EF90DF90CF90BF90AF90A0
:101690000C94D314DF91CF911F910F91FF90EF9095
:1016A000DF90CF90BF90AF900895DF92EF92FF92BE
:1016B0000F931F93CF93DF93EC017901D02E888590
:1016C0009985681779070CF047C02A853B85421732
:1016D00053070CF041C09B012E0D3F1D821793074D
:1016E0001CF47C01E61AF70A2FEF260F2E0D042FAB
:1016F000CE010E94481580913E0490913F040E94C3
:10170000D414EAA1FBA190818CA5892B8083E8A148
:10171000F9A190818BA5809589238083E114F10440
:1017200061F0612FCE010E94A6146D2DCE010E94A2
:10173000A61481E0E81AF108F1CFE8A1F9A190819F
:101740008BA5892B8083DF91CF911F910F91FF9003
:10175000EF90DF900C94D314DF91CF911F910F91F4
:10176000FF90EF90DF900895DF92EF92FF920F933A
:101770001F93CF93DF93EC017901D02E8885998553
:10178000681779070CF047C08A859B854817590769
:101790000CF041C09A012E0D3F1D821793071CF4D7
:1017A0007C01E41AF50A0FEF040F0E0D262FCE016F
:1017B0000E94481580913E0490913F040E94D414E9
:1017C000EAA1FBA190818CA5892B8083E8A1F9A1D6
:1017D00090818BA5809589238083E114F10461F0C9
:1017E000612FCE010E94A6146D2DCE010E94A61479
:1017F00081E0E81AF108F1CFE8A1F9A190818BA569
:10180000892B8083DF91CF911F910F91FF90EF90F3
:10181000DF900C94D314DF91CF911F910F91FF9023
:10182000EF90DF900895EF92FF920F931F93CF9365
:10183000DF931F92CDB7DEB77C01CB01122F77FD6E
:1018400053C0D70118966D917C9119978617970709
:101850000CF04AC057FD48C01A966D917C911B97B9
:10186000461757070CF040C001E0040F21E0280F95
:10187000682FC70139830E94481580913E049091DA
:101880003F040E94D414D7019296ED91FC91939756
:1018900090819C968C919C97892B80839096ED915A
:1018A000FC91919790819B968C9180958923808360
:1018B0003981632FC7010E94A614612FC7010E94BE
:1018C000A614D7019096ED91FC91919790819B96EB
:1018D0008C91892B80830F90DF91CF911F910F9175
:1018E000FF90EF900C94D3140F90DF91CF911F9144
:1018F0000F91FF90EF900895DC01ED91FC91019024
:10190000F081E02D09946115710579F0FB010190DA
:101910000020E9F73197AF01461B570BDC01ED9131
:10192000FC910280F381E02D099480E090E008951D
:101930004F925F926F927F92EF92FF920F931F935D
:10194000CF93DF93CDB7DEB7A1970FB6F894DEBF84
:101950000FBECDBF7C01FA01CB0119A2223008F4E1
:101960002AE08E010F5D1F4F422E512C612C712CED
:10197000BF01A30192010E948638F901CA010150FA
:1019800011096A3014F4605D01C0695CD8016C9380
:10199000232B242B252B61F7B801C7010E94830C50
:1019A000A1960FB6F894DEBF0FBECDBFDF91CF91E9
:1019B0001F910F91FF90EF907F906F905F904F90ED
:1019C00008950F931F93CF93DF93EC010E94830C34
:1019D0008C0166ED72E0CE010E94830C800F911F96
:1019E000DF91CF911F910F9108950C94830C1F925A
:1019F0000F920FB60F9211242F933F934F935F9343
:101A00006F937F938F939F93AF93BF93EF93FF93C6
:101A100081EA93E00E94E108FF91EF91BF91AF91BD
:101A20009F918F917F916F915F914F913F912F91F6
:101A30000F900FBE0F901F9018951F920F920FB628
:101A40000F9211242F938F939F93EF93FF93E09125
:101A5000B103F091B2038081E091B703F091B80334
:101A600082FD12C090818091BA038F5F8F732091A5
:101A7000BB03821751F0E091BA03F0E0EF55FC4F41
:101A8000958F8093BA0301C08081FF91EF919F9160
:101A90008F912F910F900FBE0F901F901895CF939D
:101AA000DF93282F30E0F901EA5CFF4E8491F901C1
:101AB000EE58FF4ED491F901E25AFF4EC491CC2367
:101AC00091F081110E947509EC2FF0E0EE0FFF1FDD
:101AD000EC5AFF4EA591B491EC91ED2381E090E09A
:101AE00021F480E002C080E090E0DF91CF91089582
:101AF0001F93CF93DF93282F30E0F901EA5CFF4E6C
:101B00008491F901EE58FF4ED491F901E25AFF4E4B
:101B1000C491CC23C9F0162F81110E947509EC2FB6
:101B2000F0E0EE0FFF1FE65BFF4EA591B4918FB77B
:101B3000F894111105C09C91ED2FE095E92302C0A6
:101B4000EC91ED2BEC938FBFDF91CF911F91089516
:101B5000CF93DF9390E0FC01EE58FF4E2491FC01FF
:101B6000E25AFF4E8491882361F190E0880F991F1B
:101B7000FC01EE54F54FC591D491FC01E65BFF4E9C
:101B8000A591B491611109C09FB7F89488812095FF
:101B900082238883EC912E230BC0623061F49FB7BF
:101BA000F8943881822F809583238883EC912E2BA3
:101BB0002C939FBF06C08FB7F894E8812E2B288303
:101BC0008FBFDF91CF9108958F929F92AF92BF9276
:101BD000CF92DF92EF92FF926B017C010E949E09EF
:101BE0004B015C01C114D104E104F104F1F00E9445
:101BF0009E09DC01CB0188199909AA09BB09883E15
:101C00009340A105B10570F321E0C21AD108E108A3
:101C1000F10888EE880E83E0981EA11CB11CC11447
:101C2000D104E104F10419F7DDCFFF90EF90DF90CC
:101C3000CF90BF90AF909F908F9008951F920F927A
:101C40000FB60F9211242F933F938F939F93AF93CF
:101C5000BF938091220390912303A0912403B0911C
:101C600025033091980323E0230F2D3720F40196AC
:101C7000A11DB11D05C026E8230F0296A11DB11DAF
:101C8000209398038093220390932303A09324032B
:101C9000B09325038091990390919A03A0919B039F
:101CA000B0919C030196A11DB11D8093990390935F
:101CB0009A03A0939B03B0939C03BF91AF919F9114
:101CC0008F913F912F910F900FBE0F901F901895FD
:101CD0001F920F920FB60F9211242F933F934F93A1
:101CE0005F936F937F938F939F93AF93BF93EF9384
:101CF000FF93E0919F03F091A003309709F451C046
:101D0000968DA685B785858591FF04C09C91892312
:101D100029F447C09C91892309F043C0A389B48961
:101D20009C918589809589238C93868997890197D1
:101D3000F1F7608D718DA685B785558538E020E077
:101D4000CB010197F1F7822F90E095958795282F89
:101D50004C91452309F02068315091F7868D81FD23
:101D6000209580919E0390E001968F739927309182
:101D70009D03381749F0A0919E03B0E0A85ABC4FCC
:101D80002C9380939E0303C0868D8160868F828D05
:101D9000938D0197F1F7A389B4899C918589892B4B
:101DA0008C93FF91EF91BF91AF919F918F917F9114
:101DB0006F915F914F913F912F910F900FBE0F90B8
:101DC0001F901895E0919F03F091A003E817F90781
:101DD00069F4A389B4899C918589809589238C9322
:101DE0001092A00310929F0381E0089580E008956F
:101DF0000895FC016370658B84819581268137810C
:101E0000613039F0633029F09187808733872287EA
:101E10000895318720879387828708952F923F9274
:101E20004F925F926F927F928F929F92AF92BF92EA
:101E3000CF92DF92EF92FF920F931F93CF93DF9396
:101E4000CDB7DEB76C970FB6F894DEBF0FBECDBF2F
:101E50009C8F8B8F5B011A011F830E833701C98210
:101E6000DC0158964D915C9159974115510509F047
:101E7000E5C018968D919C911997681779070CF019
:101E8000CAC11A968D919C911B97281639060CF0A1
:101E9000C2C18C2C912CFB0136E0C39EE00DF11DDC
:101EA0001124FB87EA871E161F060CF0B4C1C4017B
:101EB00033E0880F991F3A95E1F79D878C87820D53
:101EC000931D181619060CF0A6C157968C91811116
:101ED00003C0203B08F02F5FAB8DBC8DED91FC91D2
:101EE00011970284F385E02DCD012A8F09952A8D63
:101EF000B5E02B9F90011124F5013596FF87EE8701
:101F0000BB82AA822501A9014A195B09598B488B1A
:101F1000C10108969B8B8A8BE889F989E40DF51D30
:101F2000EA5CF44F9491988761013D822C82A885E8
:101F3000A0FF13C0AB8DBC8DED91FC91B981B13088
:101F400031F40484F585E02D2E813F8116C006848E
:101F5000F785E02DEE80FF801AC0EE81FF816E16BE
:101F60007F06F1F0AB8DBC8DED91FC91B981B13064
:101F700051F40484F585E02D9301A601B2018B8D07
:101F80009C8D09950DC00684F785E02D73018401B1
:101F900094014C815D816A817B818B8D9C8D09953B
:101FA000E885E695E887FFEFCF1ADF0A2C813D81AF
:101FB000280D391D3D832C834A895B89C416D506BB
:101FC00009F0B5CF5FEF451A550A8A819B81880DCC
:101FD000991D9B838A83AE85BF854A165B0609F0EF
:101FE0009BCFEE81FF816E167F0609F4F2C0EB8D68
:101FF000FC8DA081B181F981F13079F4B5016B5F7D
:102000007F4F5096ED91FC915197830128E030E08D
:10201000A1018B8D9C8D0995DCC06A857B85681933
:1020200079091E96ED91FC911F9773010C851D8512
:102030009401A1018B8D9C8D0995CBC0FA0134963A
:102040009491329765917491291BCB01B7E02B9F36
:10205000800D911D1124FA01259134913B8B2A8B1F
:10206000FC01459154915B834A83FC013296C490F4
:10207000319654915E87329614913196D49089812D
:10208000823058F0612E012E000C7708AD2D0D2CFA
:10209000000CBB0BB987A88704C019861886612C71
:1020A000712CAB8DBC8DED91FC9111970284F38561
:1020B000E02DCD010995B9818B2E912C689CC00132
:1020C000699C900D789C900D1124FC01EA0DFB1D7C
:1020D000FD87EC871C82712C612CE12F110FFF0B07
:1020E00095012E0F3F1F3B872A87AC0CB11CA50121
:1020F0004E0F5F1F5F8B4E8BC1018D0D911DD7FC65
:102100009A95998F888F4E85641608F062C0862D47
:1021100090E048855985480F591F489D9001499D79
:10212000300D589D300D1124D901A20DB31DB98B6E
:10213000A88BAA84BB844C845D84DC80BA85DB1ABE
:10214000E88DF98DE80FF91FFD8BEC8B8D2D8A0D35
:102150002E893F89A216B306B9F1877061F48A818E
:102160009B810196EA89FB89AA81BB81EA0FFB1F4B
:1021700074909B838A8377FE20C0AB8DBC8DED91DC
:10218000FC91B981B13061F40484F585E02D2E8194
:102190003F814C895D89B5018B8D9C8D09950DC062
:1021A0000684F785E02DEE80FF8084019401488944
:1021B0005989B2018B8D9C8D0995770CEFEFAE1A82
:1021C000BE0A480C591CC2CF3C813C0D3C83639431
:1021D0009ACFAB8DBC8DED91FC9111970688F78954
:1021E000E02DCD016C960FB6F894DEBF0FBECDBFCB
:1021F000DF91CF911F910F91FF90EF90DF90CF90E3
:10220000BF90AF909F908F907F906F905F904F9016
:102210003F902F9009946C960FB6F894DEBF0FBED6
:10222000CDBFDF91CF911F910F91FF90EF90DF9085
:10223000CF90BF90AF909F908F907F906F905F9066
:102240004F903F902F900895AF92BF92CF92EF9210
:10225000FF920F931F93CF93DF93EC01262F888D6E
:10226000998D009709F040C06A3059F41D861C868C
:102270002C898E859F8538E0239F800D911D112428
:1022800041C06D3009F4AAC08E898823C1F03C8911
:102290008C859D8546E0349F800D911D11244885D5
:1022A0005985481759075CF41D861C868E859F85C5
:1022B00048E0349F800D911D11249F878E87EA8806
:1022C000FB88088919894E855F856C857D85CC885A
:1022D000CE010E940E0F2C898C859D8536E0239FB0
:1022E000800D911D112442C06A3079F41D861C8630
:1022F0002C89FC013696E4918E859F852E9F800D5A
:10230000911D11249F878E8769C06D3009F466C0C6
:10231000FC0134963491631708F460C03196E4915F
:10232000E61708F45BC0FC013296A590B490462FE6
:1023300050E0431B510937E0349FB001359F700DC9
:102340001124A60EB71EF501329634913196E49110
:10235000332311F0E1110DC0F5013496E4912C897D
:102360008C859D85E29F800D911D11249D878C8712
:1023700035C0F501359644915E89552311F16C897C
:10238000E32FF0E0E40FF11D47FDFA956E9FD001B9
:102390006F9FB00D11244C855D854A0F5B1FE8854A
:1023A000F985E417F5076CF41D861C86FC0136964A
:1023B000E4918E859F856E9F800D911D11249F87CE
:1023C0008E87EA88FB88088919894E855F856C8528
:1023D0007D85CC88CE010E940E0FBECF81E090E0BB
:1023E000DF91CF911F910F91FF90EF90CF90BF9011
:1023F000AF9008956F927F928F929F92AF92BF920B
:10240000CF92DF92EF92FF920F931F93CF93DF93C0
:10241000EC014B015A0169013801E881F98102841C
:10242000F385E02D0995E881F9810288F389E02D93
:1024300087019601A501B401CE010995E881F981D2
:10244000A501460D571D415051090288F389E02D21
:102450009601B401CE010995E881F9810088F189DE
:10246000E02D9301A501B401CE010995E881F98120
:10247000C80CD91CB601615071090088F189E02DA2
:102480009301A501CE010995E881F9810688F789B4
:10249000E02DCE01DF91CF911F910F91FF90EF9032
:1024A000DF90CF90BF90AF909F908F907F906F9074
:1024B0000994CF92DF92EF92FF920F931F93CF93E5
:1024C000DF9300D000D000D0CDB7DEB76C01DC01C7
:1024D000ED91FC916217730789F4041715072CF42A
:1024E000942F852FA801092F182F041B150B980175
:1024F0002F5F3F4F048CF58DE02D12C04017510720
:1025000009F5261737072CF4962F872FB901292FA5
:10251000382F261B370B2F5F3F4F068CF78DE02D92
:102520008701C601099526960FB6F894DEBF0FBE47
:10253000CDBFDF91CF911F910F91FF90EF90DF9072
:10254000CF9008950284F385E02D2D833E834B8345
:102550005C8369837A830995D601ED91FC910488A7
:10256000F589E02D2D813E814B815C8169817A81E5
:10257000C6010995D601ED91FC910688F789E02DF9
:10258000C60126960FB6F894DEBF0FBECDBFDF9111
:10259000CF911F910F91FF90EF90DF90CF90099412
:1025A000EF92FF920F931F93DC01ED91FC91119735
:1025B0001A960D911C911B9718962D913C91199785
:1025C00000A0F1A1E02D7B0140E050E060E070E070
:1025D00009951F910F91FF90EF9008954F925F9290
:1025E0006F927F928F929F92AF92BF92CF92DF9223
:1025F000EF92FF920F931F93CF93DF9300D0CDB74D
:10260000DEB76C015A0139014801DC01ED91FC9102
:102610000284F385E02D69837A8309956981462ECA
:102620007A81572E640C751CD601ED91FC914614ED
:1026300057046CF40088F189E02D87019401A5010D
:10264000B201C6010995BFEF4B1A5B0AEDCF0688B0
:10265000F789E02DC6010F900F90DF91CF911F9168
:102660000F91FF90EF90DF90CF90BF90AF909F9031
:102670008F907F906F905F904F900994AF92BF9230
:10268000CF92DF92EF92FF920F931F93CF93DF933E
:1026900000D000D0CDB7DEB75C016901DC01ED915F
:1026A000FC910284F385E02D4B835C8369837A83FC
:1026B0000995D501ED91FC9169817A819B012C0DE1
:1026C0003D1D215031090488F589E02D78014B81A9
:1026D0005C818A01C5010995D501ED91FC910688BF
:1026E000F789E02DC5010F900F900F900F90DF91AB
:1026F000CF911F910F91FF90EF90DF90CF90BF90FF
:10270000AF900994AF92BF92CF92DF92EF92FF9277
:102710000F931F93CF93DF9300D000D0CDB7DEB7D8
:102720005C016901DC01ED91FC910284F385E02DEF
:102730004B835C8369837A830995D501ED91FC9184
:102740004B815C81C40ED51EB1E0CB1AD108048840
:10275000F589E02D7801860169817A819B01C501A7
:102760000995D501ED91FC910688F789E02DC50109
:102770000F900F900F900F90DF91CF911F910F91BD
:10278000FF90EF90DF90CF90BF90AF9009940895A5
:10279000EF92FF920F931F93DC01ED91FC9100A04B
:1027A000F1A1E02D09951F910F91FF90EF900895F1
:1027B0000F931F93DC01ED91FC91068CF78DE02DBA
:1027C00009951F910F9108950F931F93DC01ED91CF
:1027D000FC91048CF58DE02D09951F910F910895C2
:1027E000DC01ED91FC910084F185E02D09940895C0
:1027F0002F923F924F925F926F927F928F929F9211
:10280000AF92BF92CF92DF92EF92FF920F931F93FE
:10281000CF93DF9300D01F92CDB7DEB74C017B83FF
:102820006A836A01590117019801241B350B37FF90
:1028300003C0319521953109C5014A815B81841B13
:10284000950B97FF03C091958195910951E05983AC
:102850008217930714F019820BC09A2D8B2D580103
:10286000092F182F9A818B81DB82CA82C92ED82E1C
:102870008A819B81A816B9065CF49C2D8D2D680178
:10288000092F182F9A818B81BB82AA82A92EB82E7C
:102890002501AA81BB814A1A5B0A38016C187D08A0
:1028A00077FE03C0719461947108720157FE03C0F2
:1028B000BFEFEB1AFB0AF594E794C016D1061CF0A3
:1028C0000FEF1FEF1FC001E010E01CC0D401ED911D
:1028D000FC91B9810484F585E02D9101BB23C1F001
:1028E0004A815B81B601C4010995E618F708F7FE35
:1028F00004C0C00ED11EE40CF51CEA81FB813196A8
:10290000FB83EA834A815B81A416B506FCF604C00A
:10291000A6016A817B81E7CF0F900F900F90DF9126
:10292000CF911F910F91FF90EF90DF90CF90BF90CC
:10293000AF909F908F907F906F905F904F903F905F
:102940002F900895089580E090E00895FC01838D14
:10295000882339F06EBD00000DB407FEFDCF8EB5A3
:10296000089528E030E090E8A48DB58D81A5492F29
:10297000462319F04C91842B03C04C9180958423FD
:102980008C93A68DB78D4C9182A5842B8C93A68DAC
:10299000B78D4C9182A5809584238C939695215078
:1029A000310911F7089508958CBD9DBD08950F93C9
:1029B0001F93CF93DF931F92CDB7DEB78C01809129
:1029C0003E0490913F0469830E94D414D8019296EA
:1029D000ED91FC91939790819C968C919C97892B7B
:1029E00080839096ED91FC91919790819B968C912C
:1029F0008095892380836981C8010E94A614D8012B
:102A00009096ED91FC91919790819B968C91892B5A
:102A100080830F90DF91CF911F910F9108950F93B5
:102A20001F93CF93DF931F92CDB7DEB78C018091B8
:102A30003E0490913F0469830E94D414D801929679
:102A4000ED91FC91939790819C968C919C978095A9
:102A5000892380839096ED91FC91919790819B962C
:102A60008C918095892380836981C8010E94A61476
:102A7000D8019096ED91FC91919790819B968C91C5
:102A8000892B80830F90DF91CF911F910F91089533
:102A9000EF92FF920F931F93CF93DF9300D0CDB7A8
:102AA000DEB77C01162F6AE229834A830E940F1544
:102AB00060E0C7010E94D714F70185A5612F680F58
:102AC000C7010E94D71460E0C7010E94D714F70124
:102AD00085A52981622F680FC7010E94D7146BE278
:102AE000C7010E940F1560E0C7010E94D714F701CB
:102AF00086A54A81642F680FC7010E94D71460E041
:102B0000C7010E94D714F70186A5602F680FC7017F
:102B10000E94D7146CE2C7010F900F90DF91CF9104
:102B20001F910F91FF90EF900C940F1582E794E0A6
:102B30000E94E20E0E94DD1667E073E081EA93E0F6
:102B40000E94F50C6CEF82E794E00E94DC0962E0E1
:102B500070E080E090E00E94E40D8FB7F89440911F
:102B600022035091230360912403709125038FBFAA
:102B70004C505E4F6F4F7F4F409326035093270377
:102B8000609328037093290381EA93E00E94AB16B7
:102B900066ED72E081EA93E00C94830C60E070E0F3
:102BA00083E494E00C94690AEF92FF920F931F93D1
:102BB000CF93DF931F92CDB7DEB77C01FC0100817C
:102BC0001181C80169830E9419366981681719F05B
:102BD000C8010E942136C7010F90DF91CF911F914C
:102BE0000F91FF90EF9008952F923F924F925F9236
:102BF0006F927F928F929F92AF92BF92CF92DF920D
:102C0000EF92FF920F931F93CF93DF936C015B01C1
:102C1000EA0181E090E04C01841A950A6624772449
:102C2000641A750A660C771CE12CF12C822F8470D3
:102C3000582E822F8270482E822F8870382E217055
:102C4000222EEC16FD060CF073C097FC06C02197EF
:102C500082E0680E711C860C971C8FEFE81AF80A48
:102C6000C701880F991F0196880E991E5520B1F053
:102C70009801A5014C0F5D1FB7016C0D7D1D83E40C
:102C800094E00E94F0139801A7014A0D5B1DB60164
:102C90006C0F7D1F83E494E00E94F0134420B1F098
:102CA0009801A5014C1B5D0BB7016C0D7D1D83E4E4
:102CB00094E00E94F0139801A5014E195F09B60136
:102CC0006C0F7D1F83E494E00E94F0133320B1F079
:102CD0009801A7014A0D5B1DB6016C1B7D0B83E4B7
:102CE00094E00E94F0139801A5014C0F5D1FB601FE
:102CF0006E197F0983E494E00E94F013222009F406
:102D0000A0CF9801A5014E195F09B6016C1B7D0B80
:102D100083E494E00E94F0139801A5014C1B5D0B25
:102D2000B6016E197F0983E494E00E94F01389CF05
:102D3000DF91CF911F910F91FF90EF90DF90CF9097
:102D4000BF90AF909F908F907F906F905F904F90CB
:102D50003F902F900895CF92DF92EF92FF920F93C2
:102D60001F93CF93DF9377FF1DC06A017B01EC01B6
:102D70006DE20E947C0C8C0144275527BA014C1946
:102D80005D096E097F092AE0CE010E94980C800F30
:102D9000911FDF91CF911F910F91FF90EF90DF90E6
:102DA000CF9008952AE0DF91CF911F910F91FF906E
:102DB000EF90DF90CF900C94980C10928D041092AD
:102DC0008C0410928B0410928A0410928904109241
:102DD00088048DEC90E090938F0480938E04909102
:102DE0007E04963108F057C025E530E03093890421
:102DF000209388042BEC30E030938B0420938A04DA
:102E000020E930E030938D0420938C0420916800F9
:102E1000983050F031E09E3008F430E081E001C09D
:102E2000880F3A95EAF701C084E0822B809368000E
:102E3000983038F09E3040F0963148F020E030E095
:102E400008C02DE630E005C02BE630E002C02CE6DD
:102E500030E03093860420938504983030F481E08C
:102E600001C0880F9A95EAF70EC0292F30E09E30F6
:102E700018F42850310902C02E50310981E001C0F8
:102E8000880F2A95EAF78093870480918E049091A9
:102E90008F040197F1F780918C0490918D04892B18
:102EA00021F180919F039091A00324E08237920743
:102EB000E1F0009711F00E94E20E809190048E7F65
:102EC0008093900410929E0310929D0382E794E0F9
:102ED0009093A00380939F03E0918504F091860472
:102EE000908180918704892B8083089520915B04D1
:102EF00030915C04009749F0232B99F42091510400
:102F0000309152042A5F3F4F08C0232B51F020918B
:102F100051043091520426503109309352042093C9
:102F2000510490935C0480935B040895CF93DF93E6
:102F3000EC0161E085E00E94A80D209711F460E0AB
:102F400004C0CF3FD10531F461E085E0DF91CF913E
:102F50000C94780DEBE3F0E1E491E330F9F048F400
:102F6000E130B9F0E230A1F584B5806284BDC8BD1E
:102F700034C0E730E9F0E83019F1E43049F58091E8
:102F80008000806280938000D0938B00C0938A0081
:102F900024C084B5806884BDC7BD1FC080918000F7
:102FA000806880938000D0938900C093880015C00A
:102FB0008091B00080688093B000C093B3000DC0D2
:102FC0008091B00080628093B000C093B40005C0CF
:102FD000C038D1050CF0B8CFB2CFDF91CF910895B2
:102FE000CF92DF92EF92FF920F931F93CF93DF93D5
:102FF000EC012196FC011491112309F437C0FE0164
:10300000649183E494E00E940F156E01F2E0CF0E0C
:10301000D11CFE013196C4910C2F0078CF77760138
:10302000DC2FD15050F0F701649183E494E00E94CA
:10303000D714FFEFEF1AFF0AF4CFC6018C0F911DD2
:10304000EC01002389F07C019FEFE91AF90AFE01E7
:10305000649170E06F3F710511F464EF71E080E0FE
:1030600090E00E94E40DE7011150C6CFDF91CF91AF
:103070001F910F91FF90EF90DF90CF9008952F92C6
:103080003F924F925F926F927F928F929F92AF92F8
:10309000BF92CF92DF92EF92FF920F931F93CF9345
:1030A000DF9300D000D000D0CDB7DEB72C013B01BC
:1030B0005C834B8319011E830D835801B194A19445
:1030C000B108AA0CBB1C4A018A0C9B1C6801C40CE9
:1030D000D51C87019401AB01B60183E494E00E9402
:1030E000D813C301820D931D9A838983AC0141508B
:1030F00051099401B60183E494E00E94D813A20C14
:10310000B31CED81FE816E0E7F1E9501A301B201FD
:1031100083E494E00E94E4138B819C81480E591E45
:10312000B201615071099501A30183E494E00E940A
:10313000E41321E04D815E81B301C6010E94F415C4
:10314000ED81FE814E1A5F0AF1E04F1A510822E02C
:103150004D815E81B301C2010E94F415A980BA803D
:103160008D819E81A81AB90A91E0A91AB10824E0BC
:103170004D815E81B501C2010E94F41528E04D81A8
:103180005E81B501C6010E94F41526960FB6F8942B
:10319000DEBF0FBECDBFDF91CF911F910F91FF908A
:1031A000EF90DF90CF90BF90AF909F908F907F90E7
:1031B0006F905F904F903F902F9008954F925F9245
:1031C0006F927F928F929F92AF92BF92CF92DF9237
:1031D000EF92FF920F931F93CF93DF936C015B01EC
:1031E0004A0139012801E7018FE1E82EF12C89011C
:1031F0009A01AB01B60183E494E00E9459128E015A
:103200009201A301B40183E494E00E945912850164
:103210009601AE01B20183E494E00E945912DF915D
:10322000CF911F910F91FF90EF90DF90CF90BF90C3
:10323000AF909F908F907F906F905F904F90089588
:103240000F931F93CF93DF93EC01462F50E060E084
:1032500070E02AE00E94980C8C0166ED72E0CE01CD
:103260000E94830C800F911FDF91CF911F910F91CE
:103270000895CF93DF93CDB7DEB727970FB6F894B5
:10328000DEBF0FBECDBF789484B5826084BD84B5A7
:10329000816084BD85B5826085BD85B5816085BD51
:1032A00080916E00816080936E0010928100809109
:1032B0008100826080938100809181008160809391
:1032C0008100809180008160809380008091B100B6
:1032D00084608093B1008091B00081608093B000E1
:1032E00080917A00846080937A0080917A00826075
:1032F00080937A0080917A00816080937A00809137
:103300007A00806880937A001092C10060E084E0C7
:103310000E94A80D60E087E00E94A80D60E086E0B2
:103320000E94A80D61E085E00E94A80DE091B10324
:10333000F091B20382E08083E091AD03F091AE039F
:103340001082E091AF03F091B00387E68083109282
:10335000B903E091B503F091B60386E08083E09174
:10336000B303F091B403808180618083E091B30363
:10337000F091B403808188608083E091B303F09181
:10338000B403808180688083E091B303F091B4033B
:1033900080818F7D808364E170E080E090E00E9416
:1033A000E40D6EE571E081EA93E00E94E10C0E9479
:1033B000DD1664E170E080E090E00E94E40D65E5D8
:1033C00071E081EA93E00E94E10C64E170E080E04A
:1033D00090E00E94E40D109271041092700461E07C
:1033E000809168040E94A80D61E0809167040E94AA
:1033F000A80D2091670430E0F901E25AFF4EE491F4
:10340000F0E0EE0FFF1FE65BFF4E859194919093E5
:103410006404809363044091680450E0FA01E25A26
:10342000FF4E8491E82FF0E0EE0FFF1FE65BFF4EAA
:10343000859194919093660480936504F901EE5808
:10344000FF4EE491E0936E04FA01EE58FF4EE491D2
:10345000E0936F0480915E04882309F43AC01FB79B
:10346000F89480912A03811127C0E8E6F0E1849165
:10347000ECE7F0E19491E82FF0E0EE0FFF1FEE543F
:10348000F54FA591B491EC91E92321F461E08AE034
:103490000E94780D61E08AE00E94A80D8CB58061E1
:1034A0008CBD8CB580648CBD61E08DE00E94A80D60
:1034B00061E08BE00E94A80D80912A038F5F8093CA
:1034C0002A031FBF80E580933E0481E080933F0480
:1034D00049C061E080916B040E94A80D61E0809179
:1034E0006A040E94A80D80916B0490E0FC01E25AEE
:1034F000FF4EE491F0E0EE0FFF1FE65BFF4EA5915B
:10350000B491B0936204A093610420916A0430E006
:10351000F901E25AFF4EE491F0E0EE0FFF1FE65B87
:10352000FF4E459154915093600440935F04FC0119
:10353000EE58FF4E849180936D04F901EE58FF4ED2
:10354000E491E0936C049C91E82FE095E923EC93DF
:10355000E0915F04F0916004908180916C0480950B
:1035600089238083E0916304F091640490818091C9
:103570006E0480958923808380916904882321F1DA
:1035800061E00E94A80D61E0809169040E94780DBD
:1035900064EF71E080E090E00E94E40D60E08091D3
:1035A00069040E94780D64EF71E080E090E00E9471
:1035B000E40D61E0809169040E94780D64EF71E090
:1035C00080E090E00E94E40D84EF9AE00E94F01702
:1035D00087EE9AE00E94F0178CEB9AE00E94F017B9
:1035E00066E383E494E00E940F1560EC83E494E0CA
:1035F0000E94D71482E080935D048091420490E0A1
:103600000E94961760E070E083E494E00E94690AEB
:1036100063E083E494E00E94900A8FE29BE00E94C2
:10362000761781E08093570482E190E090935004F4
:1036300080934F048CE190E0909352048093510466
:1036400080EE9FEF9093560480935504909354041A
:103650008093530461E771E083E494E00E94F50CE9
:1036600083E190E09093500480934F044DE1C42E89
:10367000D12CD0925204C092510400E018EF109364
:10368000560400935504109354040093530461E7C7
:1036900071E083E494E00E94F50C84E190E0909363
:1036A000500480934F04D0925204C092510410935E
:1036B000560400935504109354040093530461E797
:1036C00071E083E494E00E94F50C68E873E180E027
:1036D00090E00E94E40D82E794E00E94E20E0E94D6
:1036E000DD166CE771E081EA93E00E94E10C6FEF78
:1036F00082E794E00E94DC0964E170E080E090E001
:103700000E94E40D82E794E00E94300A892BA1F127
:1037100082E794E00E94480A8C0168E871E081EA3F
:1037200093E00E94F50CA801012E000C660B770BAC
:1037300081EA93E00E94AB1662E070E080E090E0E6
:103740000E94E40D2091430330914403211531057B
:1037500029F410932C0300932B0307C0213031056B
:1037600021F410932E0300932D032F5F3F4F3093CE
:10377000440320934303C6CF1092440310924303A3
:1037800080E090E00E94761783E490E090935004EC
:1037900080934F048CE390E0909352048093510403
:1037A00080EE9FEF909356048093550490935404B9
:1037B0008093530481E08093570480912D0390916E
:1037C0002E03892B31F46DE871E083E494E00E94CC
:1037D000F50C80912D0390912E03019731F464E94B
:1037E00071E083E494E00E94F50C80912D039091A8
:1037F0002E03029731F468E971E083E494E00E94BB
:10380000F50C80912D0390912E03039731F46CE910
:1038100071E083E494E00E94F50C80912D03909177
:103820002E03049731F460EA71E083E494E00E948F
:10383000F50C82E390E09093500480934F0486E56A
:1038400090E0909352048093510480EE9FEF909308
:10385000560480935504909354048093530481E05C
:103860008093570480912B0390912C03019731F49E
:1038700065EA71E083E494E00E94F50C80912B03EB
:1038800090912C03029731F469EA71E083E494E0AB
:103890000E94F50C80912B0390912C03039731F437
:1038A0006FEA71E083E494E00E94F50C80912B03B1
:1038B00090912C03049731F465EB71E083E494E07C
:1038C0000E94F50C80912B0390912C03059731F405
:1038D0006DEB71E083E494E00E94F50C80912B0382
:1038E00090912C03069731F463EC71E083E494E04B
:1038F0000E94F50C80912B0390912C03449731F496
:1039000068E971E083E494E00E94F50C80912B0358
:1039100090912C03459731F46CEC71E083E494E0D2
:103920000E94F50C80912B0390912C03469731F463
:1039300064ED71E083E494E00E94F50C8FE190E087
:1039400090935604809355049093540480935304A9
:1039500081E0809357048EE190E09093500480932F
:103960004F048CE690E090935204809351046DEDE7
:1039700071E083E494E00E94F50C80E090E00E9406
:10398000761782E891E890935604809355049093BB
:103990005404809353041092500410924F0488E70B
:1039A00090E0909352048093510460EF71E083E4BF
:1039B00094E00E94F50C4091420450E060E070E019
:1039C0002AE083E494E00E94980C68EF71E083E4BD
:1039D00094E00E94F50C4091410450E060E070E0FA
:1039E0002AE083E494E00E94980C63E072E083E4B0
:1039F00094E00E94F50C4091400450E060E070E0DB
:103A00002AE083E494E00E94980C66E072E083E48C
:103A100094E00E94F50C6CED75E080E090E00E946F
:103A2000E40D0E94CE150E94961522242394312C79
:103A300030EEA32E37E0B32E84E00E944F0D082F06
:103A40008093570386E00E944F0D182F80935603F2
:103A500087E00E944F0D80935503013009F059C053
:103A6000113009F056C068E072E081EA93E00E94EC
:103A7000F50C0E94CE158DE090E090935004809359
:103A80004F0480E290E0909352048093510410938D
:103A9000570480E098EF90935604809355049093D8
:103AA0005404809353046CE172E083E494E00E9438
:103AB000F50C609142041A821982CE0101960E948F
:103AC000D415609141043A822982CE0101960E9468
:103AD000D4156091400482E090E09A838983CE01FE
:103AE00001960E94D41568EB7BE080E090E00E9494
:103AF000E40D6CE272E083E494E00E94F50C68EE61
:103B000073E080E090E00E94E40D0E94CE151093D7
:103B100004018091570381111FC0809156038130A9
:103B2000D9F4809140048F5F833019F08093400472
:103B300002C0109240040E94CE1566E970E080E059
:103B400090E00E94E40D81E08093040166E970E05A
:103B500080E090E00E94E40D80915703813009F0ED
:103B600043C08091550381113FC0809142048A5027
:103B70008B3008F483ED8093420465E372E081EAC0
:103B800093E00E94F50C6091420481EA93E00E9468
:103B900020198091420490E00E94961720914204DF
:103BA000269530E090EEE92EFF24FA940FE710E01E
:103BB0004FE750E060E070E083E494E00E94591227
:103BC00062E370E080E090E00E94E40D2091420406
:103BD000269530E0E12CF12C4FE750E060E070E0FA
:103BE00083E494E00E94591280915703813009F0D8
:103BF00041C0809155038130E9F5809141048A509C
:103C000009F487E98093410467E472E081EA93E074
:103C10000E94F50C6091410481EA93E00E94201912
:103C20008091410490E00E949617209141042695CE
:103C300030E08FE1E82EF12C0FE710E04FE750E085
:103C400060E070E083E494E00E94591262E370E067
:103C500080E090E00E94E40D20914104269530E040
:103C6000E12CF12C4FE750E060E070E083E494E059
:103C70000E94591280915503811103C08091420422
:103C800004C0813029F48091410490E00E9496178D
:103C90005090040191E0591204C5109254031092FF
:103CA000530310925203109251031092500310923A
:103CB0004F0310924E0310924A0310924B0310923E
:103CC0004C0310924D031092490310924803109236
:103CD0004703109246031092450310923903109245
:103CE0003A0310923B0310923C0310923D03109252
:103CF0003F03109241031092420310923803109236
:103D00002F031092400310923E031092350310923D
:103D1000340310923303109232031092370310923F
:103D20003603109231031092300330920301209237
:103D300002013092010120920001809140048150E3
:103D40008E3F08F4D3C284E190E0909350048093B6
:103D50004F049093520480935104509257049FE172
:103D6000C92ED12CD0925604C0925504D09254043E
:103D7000C09253046BE572E083E494E00E94E10C8E
:103D800068EC70E080E090E00E94E40D0E94CE15A7
:103D9000B0925604A0925504B0925404A0925304D9
:103DA00082E090E09093500480934F0490935204EB
:103DB000809351045092570464E672E083E494E0E7
:103DC0000E94E10C21E2622E712C709250046092EC
:103DD0004F0482E090E090935204809351045092FB
:103DE000570468E672E083E494E00E94E10C3FE14E
:103DF000E32EF12C0CE010E02FE930E040E050E041
:103E000060E070E083E494E00E94FA1128E230E080
:103E100040E050E06EE170E083E494E00E94FA112B
:103E200082E090E09093500480934F0441E1842E0F
:103E3000912C909252048092510450925704B09267
:103E40005604A0925504B0925404A09253046EE616
:103E500072E083E494E00E94E10C7092500460925E
:103E60004F0490925204809251045092570462E79A
:103E700072E083E494E00E94E10C2FE930E04FE02F
:103E800050E060E070E083E494E00E94FA1128E2E0
:103E900030E04FE050E06EE170E083E494E00E9497
:103EA000FA112EE130E04FE050E06AE570E083E483
:103EB00094E00E94FA118CE590E090935004809376
:103EC0004F04909252048092510450925704B09241
:103ED0005604A0925504B0925404A092530469E78A
:103EE00072E083E494E00E94E10C85E790E0909317
:103EF000500480934F049092520480925104509247
:103F000057046DE772E083E494E00E94E10C82E0E4
:103F100090E09093500480934F0480E290E090935F
:103F200052048093510450925704B0925604A092C8
:103F30005504B0925404A092530464E872E083E400
:103F400094E00E94E10C7092500460924F0480E271
:103F500090E0909352048093510450925704409102
:103F6000420350E060E070E02AE083E494E00E94C5
:103F7000980C68E872E083E494E00E94E10C2FE979
:103F800030E04EE150E060E070E083E494E00E94B5
:103F9000FA1128E230E04EE150E06EE170E083E497
:103FA00094E00E94FA1188E190E09093500480938D
:103FB0004F0450E3652E712C7092520460925104AC
:103FC00050925704B0925604A0925504B0925404F3
:103FD000A09253046BE872E083E494E00E94E10C49
:103FE00086E190E09093500480934F040CE310E03E
:103FF000109352040093510484E08093570460EEC0
:10400000862E99249A949092560480925504909208
:1040100054048092530461EA72E083E494E00E94C5
:10402000E10C8CE690E09093500480934F047092E2
:1040300052046092510450925704B0925604A092D8
:104040005504B0925404A09253046FE872E083E4E4
:1040500094E00E94E10C83E790E0909350048093F9
:104060004F04109352040093510485E08093570449
:104070009092560480925504909254048092530476
:1040800061EA72E083E494E00E94E10C72E4E72EBE
:10409000F12C0FE510E022E430E041E450E063E36E
:1040A00070E080E590E00E94DE18E6E4EE2EF12C50
:1040B00026E430E041E450E065E570E080E590E022
:1040C0000E94DE18909256048092550490925404F7
:1040D0008092530488E290E09093500480934F04C0
:1040E000FDE66F2E712C709252046092510412E022
:1040F0001093570461EA72E083E494E00E94E10CBB
:1041000090925604809255049092540480925304E5
:1041100084E090E09093500480934F047092520496
:10412000609251041093570461EA72E083E494E0D2
:104130000E94E10CB0925604A0925504B09254042F
:10414000A092530484E290E09093500480934F0433
:10415000A2E66A2E712C7092520460925104509221
:10416000570467E972E083E494E00E94E10C309226
:10417000500420924F047092520460925104509265
:1041800057046BE972E083E494E00E94E10C9092A2
:10419000560480925504909254048092530484E60D
:1041A00090E09093500480934F04BEE68B2E912CA8
:1041B0009092520480925104109357046FE972E078
:1041C00083E494E00E94E10CD0925604C09255041E
:1041D000D0925404C09253048BE890E09093500422
:1041E00080934F049092520480925104509257044D
:1041F00063EA72E083E494E00E94E10C85E990E0D8
:104200009093500480934F0412E7C12ED12CD0928A
:104210005204C09251045092570466EA72E083E45B
:1042200094E00E94E10C88E990E090935004809320
:104230004F0486E790E0909352048093510450928B
:10424000570468EC72E083E494E00E94E10C84E49B
:1042500090E09093500480934F048EE590E090930B
:1042600052048093510450925704B0925604A09285
:104270005504B0925404A092530468EA72E083E4B7
:1042800094E00E94E10C0FE1E02EF12C07E010E039
:1042900020E130E048E250E06AE570E08CE390E035
:1042A0000E943F188FE390E09093500480934F0456
:1042B000D0925204C092510450925704B0925604C6
:1042C000A0925504B0925404A09253046DEA72E097
:1042D00083E494E00E94E10C20E130E048E250E009
:1042E0006EE670E08CE390E00E943F18D0904004AE
:1042F00091E0D912A3C184E190E09093500480939F
:104300004F049093520480935104D09257040FE1CC
:1043100010E0109356040093550410935404009336
:10432000530464EB72E083E494E00E94E10C64EFD8
:1043300071E080E090E00E94E40D0E94CE15D092E2
:10434000570410935604009355041093540400939B
:1043500053048BE090E09093500480934F0430928C
:104360005204209251046BEB72E083E494E00E94CB
:10437000F50C1093500400934F0430925204209295
:10438000510461ED72E083E494E00E94F50C83E354
:1043900090E09093500480934F0430925204209206
:1043A00051046DEB72E083E494E00E94F50C87E425
:1043B00090E09093500480934F04309252042092E6
:1043C00051046EEE71E083E494E00E94F50C8BE5FD
:1043D00090E09093500480934F04309252042092C6
:1043E000510466E871E083E494E00E94F50C8FE6E6
:1043F00090E09093500480934F04309252042092A6
:1044000051046FEB72E083E494E00E94F50C83E8C2
:1044100090E09093500480934F0430925204209285
:10442000510461EC72E083E494E00E94F50C87E9AA
:1044300090E09093500480934F0430925204209265
:10444000510463EC72E083E494E00E94F50C04EE06
:10445000E02E08EAF02E03E010E024E130E048E02E
:1044600050E06AE070E080E090E00E943F1824E1B4
:1044700030E048E050E06AE070E08AE090E00E94BE
:104480003F1824E130E048E050E06AE070E084E169
:1044900090E00E943F1824E130E048E050E06AE0FC
:1044A00070E08EE190E00E943F1824E130E048E0A7
:1044B00050E06AE070E088E290E00E943F1824E15A
:1044C00030E048E050E06AE070E082E390E00E9473
:1044D0003F1824E130E048E050E06AE070E08CE30F
:1044E00090E00E943F1824E130E048E050E06AE0AC
:1044F00070E086E490E00E943F1824E130E048E05C
:1045000050E06AE070E080E590E00E943F1824E10E
:1045100030E048E050E06AE070E08AE590E00E9418
:104520003F1824E130E048E050E06AE070E084E6C3
:1045300090E00E943F1824E130E048E050E06AE05B
:1045400070E08EE690E00E943F1824E130E048E001
:1045500050E06AE070E088E790E00E943F1824E1B4
:1045600030E048E050E06AE070E082E890E00E94CD
:104570003F1824E130E048E050E06AE070E08CE869
:1045800090E00E943F1824E130E048E050E06AE00B
:1045900070E086E990E00E943F1880EEE82EFF244C
:1045A000FA9409E110E022E230E043E650E063E5EE
:1045B00070E083E494E00E94FA1103E010E024E04C
:1045C00030E041E650E066E570E083E494E00E946C
:1045D000FA1124E030E041E650E06EE670E083E45A
:1045E00094E00E94FA118DE290E090935004809341
:1045F0004F0483E690E09093520480935104D0924C
:1046000057048FEF97E0909356048093550490934E
:1046100054048093530465EC72E083E494E00E94B8
:10462000E10C82E080933103809330038093480350
:104630008093470380934603809345038091400411
:10464000823069F584E190E09093500480934F04A8
:10465000909352048093510481E0809357048FE13A
:1046600090E0909356048093550490935404809363
:1046700053046AEC72E083E494E00E94E10C64EF7E
:1046800071E080E090E00E94E40D0E94CE15B092AF
:104690005604A0925504B0925404A0925304109270
:1046A00004018091570381110C949330809156033B
:1046B00081110C94933082E794E00E94300A97FFB6
:1046C00002C00C94933082E794E00E94480A4C01A7
:1046D00062E070E080E090E00E94E40D81149104BB
:1046E00021F097FE02C00C94933080914303909187
:1046F00044038F30910514F00C94933001969093FD
:1047000044038093430363ED72E081EA93E00E94E7
:10471000F50C2401092C000C66087708B301A201EE
:1047200081EA93E00E94AB1662E070E080E090E0E6
:104730000E94E40D8091430390914403019709F096
:1047400021C28091540390E08815990509F41AC29A
:1047500094E5981518F08092420303C085E5809394
:1047600042038091400481115CC0E12CF12C0AE0ED
:1047700010E02DE030E04FE150E06FE170E083E4C5
:1047800094E00E94DB0AD09042036D2D70E026E594
:1047900030E0261B370B6A5B7F4F4FE150E083E42C
:1047A00094E00E94DB0A29E02D1510F00C94B6303D
:1047B00081E290E09093500480934F0480E290E077
:1047C000909352048093510481E080935704B092F7
:1047D0005604A0925504B0925404A092530494E657
:1047E000D99EA0011124052E000C660B770B83E4E3
:1047F00094E00E94AB1666ED72E083E494E00E94C0
:10480000830C2091420330E0E12C18EFF12E08E0F8
:1048100010E04FE150E067E470E083E494E00E9430
:10482000DB0A80914004813009F0ACC1E12CF12C0D
:1048300004E210E024E330E042E250E067E370E09D
:1048400083E494E00E94DB0A109142031A3010F4D2
:104850000C94BA3085E390E09093500480934F0419
:104860008EE390E0909352048093510482E0809311
:1048700057048FE29BE00E947617B0925604A092F4
:104880005504B0925404A092530424E6129FA00150
:104890001124052E000C660B770B83E494E00E9434
:1048A000AB1680E090E00E9476178091420385303D
:1048B00028F0B0EEEB2EB7E0FB2E02C0E12CF12C7D
:1048C00002E010E021E130E044E050E06CE070E014
:1048D00082E090E00E94FF32809142038A3028F00B
:1048E000A0EEEA2EA7E0FA2E02C0E12CF12C02E0A5
:1048F00010E021E130E044E050E06CE070E08CE05A
:1049000090E00E94FF32809142038F3028F0F0EE59
:10491000EF2EF7E0FF2E02C0E12CF12C02E010E0B8
:1049200021E130E044E050E06CE070E086E190E0AE
:104930000E94FF3280914203843128F0E0EEEE2E97
:10494000E7E0FE2E02C0E12CF12C02E010E021E1B4
:1049500030E044E050E06CE070E080E290E00E94E3
:10496000FF3280914203893128F070EEE72E77E024
:10497000F72E02C0E12CF12C02E010E021E130E042
:1049800044E050E06CE070E08AE290E00E94FF3288
:10499000809142038E3128F060EEE62EFF24FA94D7
:1049A00002C0E12CF12C02E010E021E130E044E013
:1049B00050E06CE070E084E390E00E94FF32809170
:1049C0004203833228F050EEE52EFF24FA9402C011
:1049D000E12CF12C02E010E021E130E044E050E075
:1049E0006CE070E08EE390E00E94FF328091420321
:1049F000883228F040EEE42EFF24FA9402C0E12C25
:104A0000F12C02E010E021E130E044E050E06CE005
:104A100070E088E490E00E94FF32809142038D3282
:104A200028F030EAE32E3DEFF32E02C0E12CF12C0A
:104A300002E010E021E130E044E050E06CE070E0A2
:104A400082E590E00E94FF3280914203823328F099
:104A500020EAE22E2DEFF22E02C0E12CF12C02E032
:104A600010E021E130E044E050E06CE070E08CE5E3
:104A700090E00E94FF3280914203873328F090EA51
:104A8000E92E9DEFF92E02C0E12CF12C02E010E09E
:104A900021E130E044E050E06CE070E086E690E038
:104AA0000E94FF32809142038C3320F0E12C88EF8A
:104AB000F82E02C0E12CF12C02E010E021E130E000
:104AC00044E050E06CE070E080E790E00E94FF324C
:104AD00080914203813420F0E12C08EFF02E02C0D7
:104AE000E12CF12C02E010E021E130E044E050E064
:104AF0006CE070E08AE790E00E94FF328091420310
:104B0000863420F0E12C18EFF12E02C0E12CF12CBC
:104B100002E010E021E130E044E050E06CE070E0C1
:104B200084E890E00E94FF32809142038B3428F0A9
:104B3000B6EBEB2EBBE8FB2E02C0E12CF12C02E021
:104B400010E021E130E044E050E06CE070E08EE8FD
:104B500090E00E94FF3280914203803528F0A6EB5E
:104B6000EA2EABE8FA2E02C0E12CF12C02E010E0B4
:104B700021E130E044E050E06CE070E088E990E052
:104B80000E94FF328091430390914403029709F001
:104B900093C08091530390E08815990509F48CC067
:104BA0008092410380914004811132C0E12CF12CAC
:104BB0000FE010E022E230E04EE650E064E670E004
:104BC00083E494E00E94DB0A80EE9FEF909356040A
:104BD00080935504909354048093530483E688157E
:104BE00018F08FE690E002C084E690E090935004C5
:104BF00080934F048EE690E090935204809351048A
:104C000082E080935704682D83E494E00E94201989
:104C100080914004813009F04FC0FFE1EF2EF12C6C
:104C200002E010E02CE130E046E250E061E670E0A6
:104C300088E290E00E943F188FEF97E0909356042F
:104C4000809355049093540480935304E12CF12CE9
:104C50000FE010E022E230E04DE650E06AE270E062
:104C600083E494E00E94DB0A80EE9FEF9093560469
:104C700080935504909354048093530440914103CE
:104C8000443618F481E390E002C08AE290E0909309
:104C9000500480934F048DE690E0909352048093EB
:104CA000510482E08093570450E060E070E02AE015
:104CB00083E494E00E94980C809143039091440314
:104CC000039709F091C08091520390E088159905EF
:104CD00009F48AC094E6981518F08092400303C046
:104CE00084E6809340038091400481117DC080EE72
:104CF0009FEF9093560480935504909354048093AF
:104D00005304E12CF12C0AE010E024E130E041E012
:104D100050E06FE170E083E494E00E94DB0A2091B0
:104D200040032B83622F70E080E090E00E944B37BD
:104D30002DE33AE047E55FE30E9400386B017C0118
:104D40009B01AC0160E070E08CEA92E40E942F3697
:104D50000E9413376C837D838E839F8320E030E035
:104D60004CE852E4C701B6010E9430360E94133766
:104D7000E12CF12C2C813D8141E050E083E494E072
:104D80000E94DB0A81E290E09093500480934F04EC
:104D900082E090E0909352048093510481E08093EC
:104DA00057046B8183E494E00E94201960914003D2
:104DB00070E080E090E00E944B372DE33AE047E559
:104DC0005FE30E9400380E941337EE24EA94E7E084
:104DD000FE2E08E010E09B0142E050E067E470E046
:104DE00083E494E00E94DB0A8091430390914403A2
:104DF000049709F018C18114910409F414C1809139
:104E00000201909103018816990609F40CC1909251
:104E10000101809200018091400481112DC0E12C9C
:104E2000F12C09E010E024E130E041E150E06BE7D3
:104E300070E083E494E00E94DB0A80EE9FEF9093A1
:104E400056048093550490935404809353048BE745
:104E500090E09093500480934F0481E190E0909310
:104E600052048093510481E080935704B301A2015E
:104E700083E494E00E94AB16909140049B839130B0
:104E800009F066C05FE1E52EF12C02E010E02CE1B4
:104E900030E046E250E061E670E080E090E00E94A1
:104EA0003F18CC24CA9467E0D62ED0925604C09204
:104EB0005504D0925404C09253043092500420926E
:104EC0004F0483E690E090935204809351042B8129
:104ED0002093570469ED72E083E494E00E94F50C9E
:104EE000E12CF12C00E110E023E230E04BE650E051
:104EF00061E070E083E494E00E94DB0A40910001ED
:104F0000509101014436510514F40C94BE3082E0F6
:104F100090E09093500480934F048DE690E090933E
:104F200052048093510480E098EF9093560480934C
:104F30005504909354048093530482E08093570463
:104F4000052E000C660B770B83E494E00E94AB16F1
:104F500080914004823009F066C03FE1E32EF12CDD
:104F600002E010E02CE130E046E250E062E070E068
:104F700080E090E00E943F18CC24CA9447E0D42EF1
:104F8000D0925604C0925504D0925404C092530457
:104F90003092500420924F0484E090E090935204A9
:104FA0008093510481E08093570469ED72E083E4BB
:104FB00094E00E94F50CE12CF12C00E110E023E2DA
:104FC00030E04CE050E061E070E083E494E00E9467
:104FD000DB0A40910001509101014436510514F45F
:104FE0000C94D43082E090E09093500480934F046E
:104FF0008EE090E0909352048093510480E098EF0B
:1050000090935604809355049093540480935304D2
:1050100082E080935704052E000C660B770B83E427
:1050200094E00E94AB16809143039091440305974E
:1050300009F094C08091510390E08815990509F416
:105040008DC0D82C80923F0380914004811127C0ED
:10505000E12CF12C0FE010E02CE030E04DE650E0C8
:1050600064E070E083E494E00E94DB0A80EE9FEF4E
:105070009093560480935504909354048093530462
:1050800084E090E09093500480934F048DE690E08C
:10509000909352048093510482E08093570480914E
:1050A0004004813039F5E12CF12C00E110E020E1E1
:1050B00030E04EE650E063E970E083E494E00E9463
:1050C000DB0A8FEF97E090935604809355049093FA
:1050D00054048093530483E990E0909350048093A8
:1050E0004F048EE690E0909352048093510482E046
:1050F0008093570480914004823039F5E12CF12CE3
:1051000009E110E022E130E044E650E066E870E0BA
:1051100083E494E00E94DB0A80EE9FEF90935604B4
:1051200080935504909354048093530486E890E050
:105130009093500480934F0484E690E0909352043F
:105140008093510483E0809357044D2D50E060E03C
:1051500070E02AE083E494E00E94980C809143037D
:10516000909144030697C1F58091500390E0881513
:10517000990591F180923E038091400481112CC0E9
:10518000E12CF12C0FE010E02CE030E04DE650E097
:1051900068E270E083E494E00E94DB0A8FEF97E01E
:1051A0009093560480935504909354048093530431
:1051B00088E290E09093500480934F048DE690E055
:1051C000909352048093510482E080935704682D99
:1051D00083E494E00E94201980914303909144035A
:1051E0000B9709F023C1C301B2010E944B372B0179
:1051F0003C019B01AC0160914A0370914B0380918B
:105200004C0390914D030E949C36882309F40EC1F3
:1052100040923A0350923B0360923C0370923D03EC
:1052200080914004811138C080EE9FEF9093560426
:10523000809355049093540480935304E12CF12CF3
:105240000AE010E02AE130E040E150E06FE170E078
:1052500083E494E00E94DB0A80E290E090935004A3
:1052600080934F0481E190E0909352048093510425
:1052700081E08093570420E030E040E251E4C30134
:10528000B2010E94A13642E00E943B3566ED72E019
:1052900083E494E00E94830C80914004813009F003
:1052A000C5C025E530E03093500420934F042CE630
:1052B00030E030935204209351048093570440907F
:1052C0003A0350903B0360903C0370903D0320E014
:1052D00030E04AEF52E4C301B2010E94FB371816D6
:1052E000BCF42FE1E22EF12C05E110E02FE130E0DB
:1052F00045E650E064E570E083E494E00E94DB0A58
:10530000B0925604A0925504B0925404A092530453
:1053100020E030E044EE52E4C301B2010E94FB37CA
:10532000181624F520E030E04CEF52E4C301B2013E
:105330000E949C3687FF1AC092E8E92E91E8F92E68
:1053400005E110E02FE130E045E650E065E570E072
:1053500083E494E00E94DB0A80EA9DEF9093560478
:1053600080935504909354048093530420E030E0DC
:1053700046EE52E4C301B2010E949C3687FF35C05D
:10538000E12C88EFF82E05E110E02FE130E045E652
:1053900050E065E570E083E494E00E94DB0A87E575
:1053A00090E09093500480934F0486E690E09093B1
:1053B00052048093510460EE72E083E494E00E9412
:1053C000F50C109256041092550410925404109249
:1053D000530485E590E09093500480934F0480E758
:1053E00090E0909352048093510420914A033091AD
:1053F0004B0340914C0350914D0360913A037091DF
:105400003B0380913C0390913D030E94303620E0A5
:1054100030E040E251E40E94A13620E030E040E07C
:105420005FE30E94003842E00E943B3580914303D5
:1054300090914403079709F0D8C080914F0390E002
:105440008815990509F4D1C0D82C80923903809130
:105450004004811127C080EE9FEF90935604809303
:1054600055049093540480935304E12CF12C0CE2E6
:1054700010E020E230E04CE350E063E770E083E4CA
:1054800094E00E94DB0A83E790E0909350048093BD
:105490004F048CE390E0909352048093510486E093
:1054A0008093570480914004813039F580EE9FEF5E
:1054B000909356048093550490935404809353041E
:1054C000E12CF12C0CE210E029E130E04CE450E05A
:1054D0006AE770E083E494E00E94DB0A8AE790E0E8
:1054E0009093500480934F048CE490E09093520486
:1054F0008093510485E0809357048091400482306A
:1055000029F5B0925604A0925504B0925404A0928A
:105510005304E12CF12C04E510E020E430E044E1F8
:1055200050E067E370E083E494E00E94DB0A87E3E5
:1055300090E09093500480934F0484E190E0909326
:105540005204809351048CE08093570498E0D91260
:1055500006C06DE872E083E494E00E94F50C80914F
:105560003903873031F46BEA72E083E494E00E94FF
:10557000F50C80913903863031F466EE72E083E4F5
:1055800094E00E94F50C80913903853031F468EE87
:1055900072E083E494E00E94F50C8091390384303A
:1055A00031F46EEE71E083E494E00E94F50C80919A
:1055B0003903833031F46DEB72E083E494E00E94B0
:1055C000F50C80913903823031F461ED72E083E4AF
:1055D00094E00E94F50C80913903813031F46BEB3B
:1055E00072E083E494E00E94F50C80914303909173
:1055F00044030897E1F580914E0390E088159905E2
:10560000B1F18092380380914004811130C080EE66
:105610009FEF909356048093550490935404809385
:105620005304E12CF12C08E110E024E130E04CE3DC
:1056300050E06CE170E083E494E00E94DB0A8CE1CE
:1056400090E09093500480934F048CE390E090930B
:1056500052048093510482E080935704482D50E017
:1056600060E070E02AE083E494E00E94980C80916E
:10567000430390914403099709F091C1882D8092CA
:10568000490310923703109236031092350310929B
:1056900034031092330310923203803228F081E0F9
:1056A0008093360380EE880D803120F091E0909356
:1056B00037038051883020F091E090933503885073
:1056C000843020F091E0909334038450823020F0B5
:1056D00091E0909333038250882319F081E0809306
:1056E00032038091400481115AC18091330381308B
:1056F00091F4C12C18EFD12E02E4E02EF12C0FE52D
:1057000010E022E430E041E450E063E370E080E543
:1057100090E00E94643380913303811120C0C12C3A
:10572000D12CA1E4EA2EF12C0EE510E021E430E0CA
:1057300040E450E064E370E080E590E00E94643370
:10574000B2E4EB2EF12C0FE510E022E430E041E46E
:1057500050E063E370E080E590E00E94DE18809105
:105760003403909147039817C1F1813091F4C12C13
:10577000E8EFDE2EF6E4EF2EF12C0FE510E026E444
:1057800030E041E450E065E570E080E590E00E94A3
:10579000643380913403811120C0C12CD12C67E483
:1057A000E62EF12C0EE510E027E430E040E450E076
:1057B00064E570E080E590E00E94643376E4E72ED3
:1057C000F12C0FE510E026E430E041E450E065E51F
:1057D00070E080E590E00E94DE18D0903503809163
:1057E00048038D1509F46AC021E0D2122BC0E12CC8
:1057F00058EFF52E07E010E020E130E048E250E0FD
:105800006AE570E08CE390E00E94FF3284E490E06F
:105810009093500480934F048EE590E0909352044F
:1058200080935104D092570410925604109255045C
:10583000109254041092530468EA72E083E494E0F6
:105840000E94E10C80913503811138C0E12CF12CCC
:1058500007E010E020E130E048E250E06AE570E067
:105860008CE390E00E94FF324FE1E42EF12C20E126
:1058700030E048E250E06AE570E08CE390E00E949E
:105880003F1884E490E09093500480934F048EE599
:1058900090E0909352048093510481E080935704E8
:1058A000B0925604A0925504B0925404A0925304AE
:1058B00068EA72E083E494E00E94E10CD090320345
:1058C000809145038D1509F46AC081E0D8122BC080
:1058D000E12C38EFF32E07E010E020E130E048E261
:1058E00050E06EE670E08CE390E00E94FF328FE3C0
:1058F00090E09093500480934F0482E790E090935F
:10590000520480935104D09257041092560410927E
:10591000550410925404109253046DEA72E083E42B
:1059200094E00E94E10C80913203811138C0E12C97
:10593000F12C07E010E020E130E048E250E06EE6B4
:1059400070E08CE390E00E94FF328FE390E0909350
:10595000500480934F0482E790E090935204809328
:10596000510481E080935704B0925604A0925504EC
:10597000B0925404A09253046DEA72E083E494E080
:105980000E94E10C2FE1E22EF12C20E130E048E210
:1059900050E06EE670E08CE390E00E943F1880914A
:1059A0004004813009F040C2809133039091460356
:1059B0009817C1F1813091F4C12C88EFD82E91E372
:1059C000E92EF12C0BE210E021E330E04DE050E055
:1059D00062E270E08CE190E00E94643380913303D6
:1059E000811120C0C12CD12C10E3E12EF12C0AE250
:1059F00010E020E330E04CE050E063E270E08CE146
:105A000090E00E94643301E3E02EF12C0BE210E001
:105A100021E330E04DE050E062E270E08CE190E0A4
:105A20000E94DE1880913403909147039817C1F1CA
:105A3000813091F4C12CA8EFDA2EB5E3EB2EF12CD6
:105A40000BE210E025E330E04DE050E064E470E06C
:105A50008CE190E00E94643380913403811120C076
:105A6000C12CD12CE6E3EE2EF12C0AE210E026E365
:105A700030E04CE050E063E470E08CE190E00E94A4
:105A80006433F5E3EF2EF12C0BE210E025E330E078
:105A90004DE050E064E470E08CE190E00E94DE189C
:105AA000D0903503809148038D1509F46AC091E0C8
:105AB000D9122BC0E12C78EFF72E07E010E020E19F
:105AC00030E04CE150E06CE470E080E090E00E9457
:105AD000FF3283E090E09093500480934F0480E580
:105AE00090E09093520480935104D0925704109206
:105AF000560410925504109254041092530468EA0C
:105B000072E083E494E00E94E10C809135038111FE
:105B100038C0E12CF12C07E010E020E130E04CE14E
:105B200050E06CE470E080E090E00E94FF326FE1B2
:105B3000E62EF12C20E130E04CE150E06CE470E026
:105B400080E090E00E943F1883E090E09093500442
:105B500080934F0480E590E0909352048093510429
:105B600081E080935704B0925604A0925504B092FD
:105B70005404A092530468EA72E083E494E00E9423
:105B8000E10CD0903203809145038D1509F46AC071
:105B900021E0D2122BC0E12C58EFF52E07E010E0E7
:105BA00020E130E04CE150E06CE470E08CE390E008
:105BB0000E94FF328FE390E09093500480934F0453
:105BC00080E590E09093520480935104D092570462
:105BD00010925604109255041092540410925304DB
:105BE0006AEE72E083E494E00E94E10C809132035B
:105BF000811138C0E12CF12C07E010E020E130E009
:105C00004CE150E06CE470E08CE390E00E94FF32E5
:105C10004FE1E42EF12C20E130E04CE150E06CE467
:105C200070E08CE390E00E943F188FE390E0909347
:105C3000500480934F0480E590E090935204809349
:105C4000510481E080935704B0925604A092550409
:105C5000B0925404A09253046AEE72E083E494E09C
:105C60000E94E10CD0903703809131038D1509F427
:105C70006AC081E0D8122BC0E12C38EFF32E07E088
:105C800010E020E130E04CE150E06CE470E08EE1A7
:105C900090E00E94FF3281E290E090935004809364
:105CA0004F0480E590E09093520480935104D09289
:105CB00057041092560410925504109254041092F6
:105CC00053046FEE72E083E494E00E94E10C809153
:105CD0003703811138C0E12CF12C07E010E020E1FE
:105CE00030E04CE150E06CE470E08EE190E00E9426
:105CF000FF322FE1E22EF12C20E130E04CE150E0C8
:105D00006CE470E08EE190E00E943F1881E290E048
:105D10009093500480934F0480E590E09093520458
:105D20008093510481E080935704B0925604A0926E
:105D30005504B0925404A09253046FEE72E083E4D1
:105D400094E00E94E10CD0903603809130038D15D1
:105D500009F46AC091E0D9122BC0E12C98EFF92E1A
:105D600007E010E020E130E04CE150E06CE470E04E
:105D70008AE590E00E94FF328DE590E09093500418
:105D800080934F0480E590E09093520480935104F7
:105D9000D092570410925604109255041092540455
:105DA0001092530464EF72E083E494E00E94E10CEB
:105DB00080913603811138C0E12CF12C07E010E00E
:105DC00020E130E04CE150E06CE470E08AE590E0E6
:105DD0000E94FF328FE1E82EF12C20E130E04CE10F
:105DE00050E06CE470E08AE590E00E943F188DE599
:105DF00090E09093500480934F0480E590E090935E
:105E000052048093510481E080935704B092560469
:105E1000A0925504B0925404A092530464EF72E02F
:105E200083E494E00E94E10C80914004823009F008
:105E30005EC180913303909146039817C1F1813080
:105E400091F4C12CA8EFDA2EB2E4EB2EF12C03E290
:105E500010E022E430E045E050E063E370E084E1EC
:105E600090E00E94643380913303811120C0C12CE3
:105E7000D12CE1E4EE2EF12C02E210E021E430E03E
:105E800044E050E064E370E084E190E00E94643319
:105E9000F2E4EF2EF12C03E210E022E430E045E0E2
:105EA00050E063E370E084E190E00E94DE188091AE
:105EB0003403909147039817C1F1813091F4C12CBC
:105EC00068EFD62E76E4E72EF12C03E210E026E40C
:105ED00030E045E050E065E570E084E190E00E944C
:105EE000643380913403811120C0C12CD12C47E44C
:105EF000E42EF12C02E210E027E430E044E050E030
:105F000064E570E084E190E00E94643356E4E52E9D
:105F1000F12C03E210E026E430E045E050E065E5D6
:105F200070E084E190E00E94DE18D090350380910B
:105F300048038D1509F46AC021E0D2122BC0E12C70
:105F400038EFF32E07E010E020E130E048E250E0C7
:105F50006AE570E080E090E00E94FF3284E490E027
:105F60009093500480934F048EE590E090935204F8
:105F700080935104D0925704109256041092550405
:105F8000109254041092530468EA72E083E494E09F
:105F90000E94E10C80913503811138C0E12CF12C75
:105FA00007E010E020E130E048E250E06AE570E010
:105FB00080E090E00E94FF322FE1E22EF12C20E100
:105FC00030E048E250E06AE570E080E090E00E9456
:105FD0003F1888E090E09093500480934F048EE542
:105FE00090E0909352048093510481E08093570491
:105FF000B0925604A0925504B0925404A092530457
:1060000068EA72E083E494E00E94E10CD0903203ED
:10601000809145038D1509F46AC081E0D8122BC028
:10602000E12C98EFF92E07E010E020E130E048E2A3
:1060300050E06EE670E080E090E00E94FF3283E086
:1060400090E09093500480934F0482E790E0909307
:10605000520480935104D092570410925604109227
:10606000550410925404109253046DEA72E083E4D4
:1060700094E00E94E10C80913203811138C0E12C40
:10608000F12C07E010E020E130E048E250E06EE65D
:1060900070E080E090E00E94FF3283E090E0909317
:1060A000500480934F0482E790E0909352048093D1
:1060B000510481E080935704B0925604A092550495
:1060C000B0925404A09253046DEA72E083E494E029
:1060D0000E94E10C8FE1E82EF12C20E130E048E253
:1060E00050E06EE670E080E090E00E943F18809102
:1060F0002F0380934903809137038093310380916C
:106100003603809330038091350380934803809158
:106110003403809347038091330380934603809137
:1061200032038093450380914303909144030C977D
:1061300009F450C040912603509127036091280331
:10614000709129032FB7F894809122039091230333
:10615000A0912403B09125032FBF481759076A0760
:106160007B07C0F10E946B090C941C1D87E290E034
:106170000C94DA238FE490E00C942C2489E090E0D6
:106180009093500480934F048DE690E090935204D6
:1061900080935104D0925604C0925504D092540476
:1061A000C09253040C949D2789E090E09093500492
:1061B00080934F048EE090E09093520480935104BA
:1061C000D0925604C0925504D0925404C092530405
:1061D0000C940828109244031092430380914203C8
:1061E0008093540380914103809353038091400333
:1061F0008093520380913F038093510380913E032B
:10620000809350038091390380934F03809138032A
:1062100080934E0380913A0390913B03A0913C03FD
:10622000B0913D0380934A0390934B03A0934C039A
:10623000B0934D038091000190910101909303016F
:106240008093020169EF72E081EA93E00E94F50C0D
:106250000E94961587CF87E491E090937304809312
:10626000720482E794E00C94E20E1092A403109260
:10627000A30388EE93E0A0E0B0E08093A5039093A1
:10628000A603A093A703B093A80329E031E03093BD
:10629000A2032093A10325EC30E03093AE032093BA
:1062A000AD0324EC30E03093B0032093AF0320EC37
:1062B00030E03093B2032093B10321EC30E030930F
:1062C000B4032093B30322EC30E03093B603209361
:1062D000B50326EC30E03093B8032093B703109257
:1062E000BA031092BB031092BC031092BD0320E5C9
:1062F00020933E0410923F0410927504109274048F
:106300008093760490937704A0937804B0937904F3
:1063100087E491E09093730480937204109289044F
:106320001092880410928B0410928A0410928D04AB
:1063300010928C0410928F0410928E04609190043D
:106340006E7F6D7F609390046695617081E0682731
:1063500083E00E94780D61E083E00E94A80DE5E7EC
:10636000F0E1E491E0938204E1E6F0E1E491F0E011
:10637000EE0FFF1FE65BFF4E85919491909384048E
:106380008093830460E082E00E94A80D80919004D5
:1063900081FD04C061E082E00E94780D82E080937C
:1063A0007E04E4E7F0E1E491E0937F04E0E6F0E1CD
:1063B000E491F0E0EE0FFF1FEC5AFF4E85919491AF
:1063C00090938104809380041092460410924504B7
:1063D00020E830E0309348042093470480EA90E0BE
:1063E00090934A048093490430934C0420934B04C7
:1063F00090934E0480934D041092580410925004D0
:1064000010924F04109252041092510481E0809334
:1064100057042FEF3FEF30935604209355043093E9
:106420005404209353048093590410925A041092F8
:106430005C0410925B042BE131E030934404209320
:1064400043049AE09093670498E09093680499E07D
:106450009093690480935E0410926B0410926A0416
:1064600080E090E00E9419368093420481E090E041
:106470000E9419368093410482E090E00E94193610
:106480008093400408952F923F924F925F926F92B3
:106490007F928F929F92AF92BF92CF92DF92EF92B4
:1064A000FF920F931F93CF93DF9300D000D000D0C3
:1064B000CDB7DEB75C014B015E834D83280181E0DF
:1064C00090E03C01641A750ACA0191958195910981
:1064D000AC01440F551F5A8349831801CC24C3943F
:1064E000D12C522F51705B8322702C83C6010197EF
:1064F0002D813E81821793070CF068C077FC0CC099
:106500008D819E8101979E838D83E981FA813296E8
:10651000FA83E9836E0E7F1EC601880F991F0196CC
:10652000680E791EFB81FF2319F12D813E81220F18
:10653000331F2F5F3F4F240D351D8701A4018D812F
:106540009E81481B590BB6016A0D7B1D83E494E0C4
:106550000E94E41391012D5F3F4FA4014C195D0986
:106560006D817E816A0D7B1D83E494E00E94E413BB
:106570009C81992321F12D813E81220F331F2F5FB2
:106580003F4F240D351D8701A401ED81FE814E1B77
:106590005F0BB5016C197D0983E494E00E94E4135C
:1065A00091012D5F3F4FA4014C195D09B5018D810B
:1065B0009E81681B790B83E494E00E94E4139FEFB3
:1065C000C91AD90AE2E02E0E311C90CF26960FB6DA
:1065D000F894DEBF0FBECDBFDF91CF911F910F9119
:1065E000FF90EF90DF90CF90BF90AF909F908F90F3
:1065F0007F906F905F904F903F902F9008952F92D3
:106600003F924F925F926F927F928F929F92AF9242
:10661000BF92CF92DF92EF92FF920F931F93CF938F
:10662000DF9300D000D0CDB7DEB72C015B011A019B
:106630003901680188279927801B910B9C01220F43
:10664000331F3C832B83C201800F911F9A83898360
:10665000240F351F8301AB01BC0183E494E00E9449
:10666000C813EB81FC816E0E7F1EF1E06F1A71087A
:10667000AC0CBD1C420C531CC2018C199D0983013A
:1066800021E0A601B50101970E94433222E0A60154
:10669000B50189819A810E9443320F900F900F902B
:1066A0000F90DF91CF911F910F91FF90EF90DF90AE
:1066B000CF90BF90AF909F908F907F906F905F90A2
:1066C0004F903F902F9008952F923F924F925F925C
:1066D0006F927F928F929F92AF92BF92CF92DF92F2
:1066E000EF92FF920F931F93CF93DF93CDB7DEB757
:1066F000AC970FB6F894DEBF0FBECDBF9CA78BA79B
:106700003B015A014901B801DC8ACB8A26153705BD
:1067100084F4892DE614F7040CF08BC14701730152
:10672000622E782E8B2D58016BA57CA54BA78CA7CC
:106730000DC0E216F306C4F4982D892D4701E92E09
:10674000F82E9A2D8B2D5B01692F782F86149704D4
:106750005CF4962D872D3401892E982E9BA58CA54F
:10676000BCA6ABA6A92EB82E6E147F0449F52BA5A6
:106770003CA5A216B3065CF09BA58CA52A153B058B
:1067800014F49A2D8B2DABA4BCA49BA78CA76A15DF
:106790007B0544F04BA55CA54617570714F47CA76E
:1067A0006BA7B5012BA53CA5261B370B2F5F3F4FD1
:1067B0000B891C89A30183E494E00E94D81342C191
:1067C000C501ABA5BCA58A1B9B0B940126193709F3
:1067D000FB01EA1BFB0BFC83EB83A701461957095E
:1067E00058874F83DB01AA19BB09BC87AB87F70128
:1067F000E819F909FE8BED8B8E149F0431F0A4018A
:10680000415051095A8F498F02C09A8E898E630177
:10681000212C312C21011F86188A198A1A8AA90174
:10682000330F660B770B4B8F5C8F6D8F7E8F2F81B5
:106830003885032E000C440B550B2F8F38A349A32A
:106840005AA3AC01990F660B770B4BA35CA36DA306
:106850007EA36B817C81072E000C880B990B6FA3A4
:1068600078A789A79AA7A98DBA8DAC15BD050CF498
:1068700051C06F85788989899A892B8D3C8D4D8D82
:106880005E8D0E94A8388BA59CA5820F931F9A83CA
:106890008983C201B1012F8D38A149A15AA10E945B
:1068A000A838ABA5BCA52A0F3B1F4F85588969891D
:1068B0007A898BA19CA1ADA1BEA1480F591F6A1F67
:1068C0007B1F4F87588B698B7A8B4FA158A569A581
:1068D0007AA5240E351E461E571E69817A81261719
:1068E000370734F499818A813A832983292F382FF5
:1068F00089819A81281B390B2F5F3F4F0B891C8997
:10690000A601BC0183E494E00E94D8139FEFC91A4A
:10691000D90AA9CFC60188199909EB85FC85E89F9A
:106920001001E99F300CF89F300C1124032C000C4F
:1069300044085508C601861997092B813C81289F78
:106940003001299F700C389F700C1124072C000C0B
:10695000880899084D895E89052E000C660B770B17
:106960004D8B5E8B6F8B788F6F817885072E000C37
:10697000880B990B6F83788789879A87CF01092EB7
:10698000000CAA0BBB0B8B879C87AD87BE87032EA1
:10699000000C440B550B2B833C834D835E83EC141E
:1069A000FD040CF44FC0C201B1012D893E894F890D
:1069B000588D0E94A838B501620F731F7A836983CE
:1069C000C401B3012F81388549855A850E94A838B2
:1069D0008BA59CA5280F391F4B855C856D857E8511
:1069E000240E351E461E571E6B817C818D819E8133
:1069F000660E771E881E991E89819A81281739078D
:106A000034F499818A813A832983292F382FA981E7
:106A1000BA812A1B3B0B2F5F3F4F0B891C89A601B4
:106A2000BD0183E494E00E94D813BFEFCB1ADB0AC8
:106A3000B6CF4301622E782E8B2DABA4BCA44BA7FE
:106A40008CA792CEAC960FB6F894DEBF0FBECDBF2A
:106A5000DF91CF911F910F91FF90EF90DF90CF903A
:106A6000BF90AF909F908F907F906F905F904F906E
:106A70003F902F9008954F925F926F927F928F92E6
:106A80009F92AF92BF92CF92DF92EF92FF926B01F3
:106A90007C01B42E9B01AC010E946D38882319F053
:106AA00065E173E027C026013701E89477F82FEFFE
:106AB0003FEF4FE75FE7C301B2010E946D388111DC
:106AC0000DC02FEF3FEF4FE75FE7C301B2010E9418
:106AD0009C3618161CF469E173E00CC02FEF3FEFF1
:106AE0004FE75FE4C701B6010E94FB37181694F424
:106AF0006DE173E083E494E0FF90EF90DF90CF903E
:106B0000BF90AF909F908F907F906F905F904F90CD
:106B10000C94830C2FEF3FEF4FE75FECC701B601FA
:106B20000E949C3687FDE4CF20E030E0A901C70138
:106B3000B6010E949C3687FF0BC06DE283E494E0AF
:106B40000E947C0C4C01F7FAF094F7F8F09402C024
:106B5000812C912CA12C60E070E080E09FE3AB14CD
:106B600041F020E030E040E251E40E94A136A394DD
:106B7000F6CF9B01AC01C701B6010E9430362B0154
:106B80003C010E941A376B017C010E9449379B012E
:106B9000AC01C301B2010E942F362B013C012AE057
:106BA000B701A60183E494E00E94980C7C01E80CF4
:106BB000F91CBB2039F06EE283E494E00E947C0C67
:106BC000E80EF91EDB2CDD2031F120E030E040E260
:106BD00051E4C301B2010E9400382B013C010E9424
:106BE0001A374B01A12CB12C2AE0B501A40183E492
:106BF00094E00E94980CE80EF91EC501B4010E94B1
:106C000049379B01AC01C301B2010E942F362B0111
:106C10003C01DA94D8CFC701FF90EF90DF90CF907E
:106C2000BF90AF909F908F907F906F905F904F90AC
:106C30000895F999FECF92BD81BDF89A992780B544
:106C40000895262FF999FECF1FBA92BD81BD20BDB0
:106C50000FB6F894FA9AF99A0FBE01960895505813
:106C6000BB27AA270E9447360C94C1370E94B3372E
:106C700038F00E94BA3720F039F49F3F19F426F417
:106C80000C94B0370EF4E095E7FB0C94AA37E92F8B
:106C90000E94D23758F3BA17620773078407950723
:106CA00020F079F4A6F50C94F4370EF4E0950B2E51
:106CB000BA2FA02D0B01B90190010C01CA01A0014E
:106CC0001124FF27591B99F0593F50F4503E68F1A9
:106CD0001A16F040A22F232F342F4427585FF3CFEA
:106CE000469537952795A795F0405395C9F77EF4BB
:106CF0001F16BA0B620B730B840BBAF09150A1F004
:106D0000FF0FBB1F661F771F881FC2F70EC0BA0F89
:106D1000621F731F841F48F4879577956795B79511
:106D2000F7959E3F08F0B0CF9395880F08F099270C
:106D3000EE0F9795879508950E94863708F481E0B5
:106D400008950E94B5360C94C1370E94BA3758F0A6
:106D50000E94B33740F029F45F3F29F00C94AA3722
:106D600051110C94F5370C94B0370E94D23768F368
:106D70009923B1F3552391F3951B550BBB27AA27F4
:106D800062177307840738F09F5F5F4F220F331F2E
:106D9000441FAA1FA9F335D00E2E3AF0E0E832D0F6
:106DA00091505040E695001CCAF72BD0FE2F29D0F9
:106DB000660F771F881FBB1F261737074807AB07CB
:106DC000B0E809F0BB0B802DBF01FF2793585F4F40
:106DD0003AF09E3F510578F00C94AA370C94F537A1
:106DE0005F3FE4F3983ED4F3869577956795B79522
:106DF000F7959F5FC9F7880F911D9695879597F92D
:106E00000895E1E0660F771F881FBB1F62177307A5
:106E10008407BA0720F0621B730B840BBA0BEE1FBA
:106E200088F7E09508950E941A376894B1110C9480
:106E3000F53708950E94DA3788F09F5798F0B92FF8
:106E40009927B751B0F0E1F0660F771F881F991F9F
:106E50001AF0BA95C9F714C0B13091F00E94F43716
:106E6000B1E008950C94F437672F782F8827B85F26
:106E700039F0B93FCCF3869577956795B395D9F7F7
:106E80003EF490958095709561957F4F8F4F9F4F01
:106E90000895E89409C097FB3EF49095809570950D
:106EA00061957F4F8F4F9F4F9923A9F0F92F96E956
:106EB000BB279395F695879577956795B795F111CB
:106EC000F8CFFAF4BB0F11F460FF1BC06F5F7F4F68
:106ED0008F4F9F4F16C0882311F096E911C077237A
:106EE00021F09EE8872F762F05C0662371F096E883
:106EF000862F70E060E02AF09A95660F771F881F52
:106F0000DAF7880F9695879597F90895990F0008F5
:106F1000550FAA0BE0E8FEEF16161706E807F9076B
:106F2000C0F012161306E407F50798F0621B730B06
:106F3000840B950B39F40A2661F0232B242B252B87
:106F400021F408950A2609F4A140A6958FEF811D2A
:106F5000811D089597F99F6780E870E060E00895CB
:106F60009FEF80EC089500240A9416161706180661
:106F70000906089500240A9412161306140605063D
:106F80000895092E0394000C11F4882352F0BB0FCE
:106F900040F4BF2B11F460FF04C06F5F7F4F8F4F31
:106FA0009F4F089557FD9058440F551F59F05F3F6C
:106FB00071F04795880F97FB991F61F09F3F79F01B
:106FC00087950895121613061406551FF2CF46959D
:106FD000F1DF08C0161617061806991FF1CF86951F
:106FE0007105610508940895E894BB276627772703
:106FF000CB0197F908950E94863708F48FEF089522
:107000000E9413380C94C1370E94B33738F00E94A5
:10701000BA3720F0952311F00C94AA370C94B037AE
:1070200011240C94F5370E94D23770F3959FC1F369
:10703000950F50E0551F629FF001729FBB27F00D26
:10704000B11D639FAA27F00DB11DAA1F649F66277B
:10705000B00DA11D661F829F2227B00DA11D621FCA
:10706000739FB00DA11D621F839FA00D611D221F84
:10707000749F3327A00D611D231F849F600D211D68
:10708000822F762F6A2F11249F5750409AF0F1F0EB
:1070900088234AF0EE0FFF1FBB1F661F771F881F54
:1070A00091505040A9F79E3F510580F00C94AA37AB
:1070B0000C94F5375F3FE4F3983ED4F386957795CB
:1070C0006795B795F795E7959F5FC1F7FE2B880FFA
:1070D000911D9695879597F908950E948637880B9C
:1070E000990B089597FB072E16F4009407D077FDAF
:1070F00009D00E94C73807FC05D03EF490958195D1
:107100009F4F0895709561957F4F0895A1E21A2EC3
:10711000AA1BBB1BFD010DC0AA1FBB1FEE1FFF1F3B
:10712000A217B307E407F50720F0A21BB30BE40B8B
:10713000F50B661F771F881F991F1A9469F76095D2
:107140007095809590959B01AC01BD01CF0108958C
:10715000052E97FB1EF400940E94BF3857FD07D000
:107160000E94863807FC03D04EF40C94BF3850952B
:107170004095309521953F4F4F4F5F4F0895909523
:107180008095709561957F4F8F4F9F4F0895AA1BF3
:10719000BB1B51E107C0AA1FBB1FA617B70710F002
:1071A000A61BB70B881F991F5A95A9F78095909534
:1071B000BC01CD010895EE0FFF1F0590F491E02D65
:1071C000099481E090E0F8940C94E63818E0C4E467
:1071D000D8E004C0FE010E94DB382196C534D107F7
:0671E000C9F7F894FFCF8F
:1071E60001000100010000000002096F089A084929
:1071F60009CB08A908BD080000000024116F08A3E8
:1072060014A214130CF713F013C813E413D813F8CD
:1072160013C713900A890AB40B550BDB0A690A597E
:1072260012FA1100000000DC096F08A314DB093014
:107236000A480AC309536F667477617265205365FD
:107246007269616C20506F7274204F70656E656450
:107256000053706974726F6E6963730053656E6470
:10726600696E6720323535003A202009004E6F4995
:107276006E697400454355005443550043414D0023
:107286005448785700454D5500546974616E005650
:10729600656E7573004D65726375727900506C7515
:1072A600746F004D65726375727932004E65707445
:1072B600756E65004E657074756E6532004469734F
:1072C600706C617920556E69742076302E313400E9
:1072D6006461796C75783A00206E696768746C75BC
:1072E600783A002028002900536176696E6720737A
:1072F600657474696E67732E2E2E2000536176694D
:107306006E672073657474696E677300202D204460
:107316006F6E6521006461796C757820736574748D
:10732600696E67733A20006E696768746C757820B9
:1073360073657474696E67733A200053637265658A
:107346006E2030005450530030302020250042413A
:107356005400202020202056004F494C0020202099
:107366002027430052504D003030004D415000530D
:107376006869667465720053656C00437572002017
:107386002020006B6D002F004C6F7752004C6F630E
:107396006B55700053637265656E2031003300369D
:1073A60000370038006B6D2F680053637265656E99
:1073B600203200093A000D0A004F696C202743006D
:1073C6004C4F572121004E0044004C6B5570004F26
:1073D600447276003247725300200950617373205D
:1073E6004D6164653A200053656E64696E672032AC
:1073F6003532202D006E616E00696E66006F76660E
:02740600000084
:00000001FF
